:100000000C940C0F0C94320F0C94320F0C94320F92
:100010000C94320F0C94320F0C94320F0C94320F5C
:100020000C94320F0C94320F0C9436120C94320F45
:100030000C94320F0C94320F0C94320F0C94320F3C
:100040000C94320F0C94320F0C94320F0C94320F2C
:100050000C94320F0C94320F0C94AB110C94320FA1
:100060000C94320F0C94320F0C94320F0C94320F0C
:100070000C94320F0C94320F0C94320F0C94320FFC
:100080000C94320F0C94320F0C94320F0C94320FEC
:100090000C94320F0C94320F0C94320F0C94320FDC
:1000A0000C94320F0C94320F0C94320F0C94320FCC
:1000B0000C94320F0C94320F0C94320F0C94320FBC
:1000C0000C94320F0C94320F0C94320F0C94320FAC
:1000D0000C94320F0C94320F0C94320F0C94320F9C
:1000E0000C94320F0C94320F0C94320F0C94320F8C
:1000F0000C94320F0C94320F0C94320F0C94320F7C
:100100000C94320F0C94320F0C94320F0C94320F6B
:100110000C94320F0C94320F0C94320F0C94320F5B
:100120000C94320F0C94320F0C94320F0C94320F4B
:100130000C94320F0C94320F0C94320F0C94320F3B
:100140000C94320F0C94320F0C94320F0C94320F2B
:100150000C94320F0C94320F0C94320F0C94320F1B
:100160000C9479110C94320F0C94320F0C94320FC2
:100170000C94320F0C94320F0C94320F0C94320FFB
:100180000C94320F0C94320F0C94320F0C94320FEB
:100190000C94320F0C94320F0C94320F0C94320FDB
:1001A0000C94320F0C94320F0C94320F0C94320FCB
:1001B0000C94320F0C94320F0C94320F0C94320FBB
:1001C0000C94320F0C94320F0C94320F0C94320FAB
:1001D0000C94320F0C94320F0C94320F0C94320F9B
:1001E0000C94320F0C94320F0C94320F0C94320F8B
:1001F0000C94320F4C696E65206E756D62657220CD
:100200006F7574206F662072616E67650000000074
:1002100000000000000000000000000053796E7430
:100220006178206572726F720000000000000000AB
:1002300000000000000000000000000000000000BE
:1002400000000000496E76616C6964206578707208
:10025000657373696F6E000000000000000000000D
:10026000000000000000000000000000556E626108
:100270006C616E63656420706172656E730000006E
:10028000000000000000000000000000000000006E
:1002900000000000446174612074797065206D690C
:1002A000736D6174636800000000000000000000CE
:1002B000000000000000000000000000496C6C65B8
:1002C00067616C206F70657261746F72000000006E
:1002D000000000000000000000000000000000001E
:1002E00000000000496C6C6567616C207661726982
:1002F00061626C650000000000000000000000006A
:10030000000000000000000000000000496C6C6567
:1003100067616C20746F6B656E2028696E746572FE
:100320006E616C206572726F72290000000000001F
:10033000000000004F7574206F66206D656D6F7250
:100340007900000000000000000000000000000034
:10035000000000000000000000000000496E74650D
:10036000676572206F766572666C6F7700000000BB
:10037000000000000000000000000000000000007D
:1003800000000000496E76616C6964206865782021
:10039000646967697400000000000000000000004C
:1003A0000000000000000000000000004865782008
:1003B0006E756D626572206F766572666C6F770020
:1003C000000000000000000000000000000000002D
:1003D000000000004D697373696E672071756F745A
:1003E00065000000000000000000000000000000A8
:1003F000000000000000000000000000457870656B
:1004000063746564206F70656E206F7220636C6F1B
:10041000736520706172656E0000000000000000CE
:1004200000000000274F4E272073796E74617820FA
:100430006572726F72000000000000000000000092
:100440000000000000000000000000004D69737310
:10045000696E67205448454E20696E2049462073D6
:10046000746174656D656E7400000000000000002A
:10047000000000004D697373696E6720544F206956
:100480006E20464F522073746174656D656E740002
:100490000000000000000000000000004C696E65D4
:1004A000206E756D626572206572726F7200000059
:1004B000000000000000000000000000000000003C
:1004C00000000000496C6C6567616C2064617461B8
:1004D000207479706500000000000000000000003A
:1004E000000000000000000000000000457870726D
:1004F000657373696F6E20746F6F20636F6D706CBE
:10050000657800000000000000000000000000000E
:10051000000000004D697373696E6720636F6D6D35
:10052000610000000000000000000000000000006A
:100530000000000000000000000000004D6973731F
:10054000696E6720636F6D6D61206F722073656DDA
:1005500069636F6C6F6E0000000000000000000017
:10056000000000004D61746820737461636B206F3C
:10057000766572666C6F7700000000000000000076
:10058000000000000000000000000000556E6469DB
:100590006D656E73696F6E6564206172726179005A
:1005A000000000000000000000000000000000004B
:1005B00000000000537562736372697074206F7578
:1005C00074206F662072616E676500000000000095
:1005D000000000000000000000000000446976698F
:1005E0006465206279207A65726F00000000000067
:1005F00000000000000000000000000000000000FB
:10060000000000004C696E65206E6F7420666F7587
:100610006E64000000000000000000000000000008
:10062000000000000000000000000000546F6F2078
:100630006D616E79206E657374656420474F535504
:1006400042730000000000000000000000000000F5
:100650000000000052455455524E20776974686F6F
:10066000757420474F535542000000000000000001
:10067000000000000000000000000000546F6F2028
:100680006D616E7920616374697665205748494CC5
:1006900045730000000000000000000000000000A2
:1006A00000000000454E44574820776974686F7514
:1006B00074205748494C450000000000000000002D
:1006C0000000000000000000000000004F4E20610C
:1006D0007267756D656E74206D7573742062652028
:1006E0003E207A65726F00000000000000000000EC
:1006F000000000004E6F6E737562736372697074F0
:10070000207661726961626C6520696E2044494D92
:100710000000000000000000000000005661726947
:1007200061626C6520616C72656164792044494D39
:10073000656E73696F6E6564000000000000000064
:1007400000000000546F6F206D616E79206163744A
:1007500069766520464F522D4E455854206C6F6F78
:100760007073000000000000000000004E45585467
:1007700020646F6573206E6F74206D6174636820F0
:10078000464F520000000000000000000000000082
:100790000000000043616E277420434F4E54696E81
:1007A000756500000000000000000000000000006F
:1007B0000000000000000000000000004F757420E1
:1007C0006F66206461746120696E20524541442047
:1007D0006F7220524553544F5245000000000000F4
:1007E000000000004E65676174697665207375626C
:1007F000736372697074206E6F7420616C6C6F77B4
:10080000656400000000000000000000496C6C6599
:1008100067616C20454550282920617267756D65B8
:100820006E740000000000000000000000000000E6
:10083000000000004F6E6C7920616C6C6F7765640E
:1008400020696E205052494E542073746174656D56
:10085000656E7400000000000000000041726775C2
:100860006D656E74206F7574206F662072616E679F
:100870006520696E20544142000000000000000025
:1008800000000000546F6F206D616E792061726707
:10089000756D656E747320696E2043414C4C000089
:1008A00000000000000000000000000041727567B9
:1008B0006D656E7420746F2074696D65242829201D
:1008C000697320756E6B6E6F776E0000000000001C
:1008D000000000002D2D203435202D2D00000000BB
:1008E0000000000000000000000000000000000008
:1008F0000000000000000000000000002D2D20344A
:1009000036202D2D00000000000000000000000037
:1009100000000000000000000000000000000000D7
:10092000000000002D2D203437202D2D0000000068
:1009300000000000000000000000000000000000B7
:100940000000000000000000000000002D2D2034F9
:1009500038202D2D000000000000000000000000E5
:100960000000000000000000000000000000000087
:10097000000000002D2D203439202D2D0000000016
:100980000000000000000000000000000000000067
:100990000000000000000000000000002D2D2035A8
:1009A00030202D2D0000000000000000000000009D
:1009B0000000000000000000000000000000000037
:1009C000000000002D2D203531202D2D00000000CD
:1009D0000000000000000000000000000000000017
:1009E0000000000000000000000000002D2D203558
:1009F00032202D2D0000000000000000000000004B
:100A000000000000000000000000000000000000E6
:100A1000000000002D2D203533202D2D000000007A
:100A200000000000000000000000000000000000C6
:100A30000000000000000000000000002D2D203507
:100A400034202D2D000000000000000000000000F8
:100A50000000000000000000000000000000000096
:100A6000000000004E6F7420656E6F75676820454A
:100A70004550524F4D20666F7220736176650000BD
:100A800000000000000000000000000053746163DB
:100A90006B20756E646572666C6F770000000000F5
:100AA0000000000000000000000000000000000046
:100AB000000000005573657220656E746572656490
:100AC00020425245414B00000000000000000000A1
:100AD00000000000000000000000000043616E27DD
:100AE00074207573652041444452207769746820EE
:100AF000636F6E7374616E7400000000000000008C
:100B0000000000004E6F7420656E6F756768206688
:100B10006C61736820666F722073617665000000F7
:100B200000000000000000000000000020000000A5
:100B300000000000000000000000000000000000B5
:100B400000000000000000000000000000000000A5
:100B50000000000000002000000000000000000075
:100B60004E2263687224000000000000424373714B
:100B70007274000000000000A9446162730000006C
:100B800000000000E542726E6400000000000000FA
:100B90007A4473676E0000000000000059227461FF
:100BA00062000000000000000000200000000000C3
:100BB000000000005A447065656B000000000000F2
:100BC0001B4465657000000000000000022268659B
:100BD000780000000000000000002000000000007D
:100BE0000000000043226865783200000000000029
:100BF0002822686578340000000000003D447065DC
:100C0000656B3136000000001F447065656B333240
:100C1000000000007744616464720000000000007E
:100C200017446565703136000000000013446565A7
:100C300070333200000000000000200000000000BF
:100C400000000000FF206C65740000000000000040
:100C5000FF2000000000000000000000642270720D
:100C6000696E7400000000009D26666F720000002F
:100C70000000000064246E6578740000000000002D
:100C8000D12174726F6E000000000000D5217472D3
:100C90006F66660000000000AF1F706F6B6500009C
:100CA00000000000FF2264696D00000000000000E9
:100CB0004D1F72656D000000000000000000200064
:100CC0000000000000000000591F64617461000012
:100CD000000000002726726561640000000000002B
:100CE000A923726573746F72650000000000676F5E
:100CF0007375620000000000000028000000000082
:100D000000000000000029000000000000000000BA
:100D1000A620676F746F000000000000AE1F6F6EAA
:100D20000000000000000000971F72657475726E6D
:100D3000000000003A256966000000000000000085
:100D40005526696E7075740000000000822073746F
:100D50006F700000000000001F20656E640000003E
:100D60000000000032207768696C65000000000018
:100D7000B01F656E64776800000000003625656569
:100D800070000000000000003225656570313600FB
:100D9000000000002E256565703332000000000061
:100DA0000000200000000000000000000000200003
:100DB00000000000000000000741616E64000000B8
:100DC0000000000029416F720000000000000000D8
:100DD0004B41656F72000000000000004424696E02
:100DE000627974650000000000002000000000002F
:100DF000000000009B236F6E74696D6500000000A9
:100E00009C236F6E69727100000000009D23726563
:100E100074690000000000009E236F6E70616363C0
:100E200000000000D821736C6565700000000000B0
:100E30000000200000000000000000000000200072
:100E40000000000000000000000020000000000082
:100E50000000000000002000000000000000000072
:100E60000000200000000000000000000000200042
:100E7000000000000000000047403C0000000000AF
:100E8000000000001B403E000000000000000000C9
:100E9000EF3F3C3D0000000000000000C33F3E3D2E
:100EA0000000000000000000973F3D00000000002F
:100EB000000000006B3F3C3E00000000000000000E
:100EC0000000200000000000000000000000746F1F
:100ED000000000000000000000007468656E000063
:100EE000000000000000656C736500000000000059
:100EF0000000737465700000000000000000200016
:100F000000000000000000000000200000000000C1
:100F100000000000000020000000000000000000B1
:100F20000000200000000000000000000000200081
:100F30000000000000000000E5402B000000000061
:100F400000000000C3402D00000000000000000071
:100F500000002B00000000000000000064223F00A1
:100F600000000000000000004D1F270000000000EE
:100F70000000000000002000000000000000000051
:100F80000000200000000000000000000000200021
:100F90000000000000000000000020000000000031
:100FA0000000000000002000000000000000000021
:100FB00000002000000000000000000000002000F1
:100FC0000000000000000000000020000000000001
:100FD00000000000000020000000000000000000F1
:100FE00000002000000000000000000000002000C1
:100FF000000000000000000073402A000000000014
:101000000000000074412F000000000000000000FC
:101010009B406D6F64000000000000000000200095
:1010200000000000000000000000200000000000A0
:101030000000000000002000000000000000000090
:101040000000200000000000000000000000200060
:101050000000000000000000000020000000000070
:101060000000000000002000000000000000000060
:101070000000200000000000000000000000200030
:101080000000000000000000000020000000000040
:101090000000000000002000000000000000000030
:1010A0000000200000000000000000000000200000
:1010B0000000000000000000003F5E000000000093
:1010C0000000000000002000000000000000000000
:1010D00000002000000000000000000000002000D0
:1010E00000000000000000000000200000000000E0
:1010F00000000000000020000000000000000000D0
:10110000000020000000000000000000000020009F
:1011100000000000000000000000200000000000AF
:10112000000000000000200000000000000000009F
:10113000000020000000000000000000000020006F
:10114000000000000000000000002000000000007F
:10115000000000000000200000000000000000006F
:10116000000020000000000000000000000020003F
:101170000000000000000000713E40000000000080
:1011800000000000C13E6E6F74000000000000000F
:10119000DE3E2D000000000000000000293E40332C
:1011A0003200000000000000993E4031360000008F
:1011B000000000000000200000000000000000000F
:1011C00000002000000000000000000000002000DF
:1011D00000000000000000000000230000000000EC
:1011E0000000000000003D000000000000000000C2
:1011F00030363A00000000000000000000003B0014
:10120000000000000000000000002C0000000000B2
:1012100000000000000020000000000000000000AE
:10122000000020000000000000000000000020007E
:101230000000000000000000656573697A65000029
:101240000000000000000000080000000000000096
:1012500000000000000000000000000000007469B1
:101260006D657230000000000000000000F0FF0417
:1012700074696D657231000000000000000000F12B
:10128000FF0474696D657232000000000000000008
:1012900000F2FF0474696D65723300000000000005
:1012A000000000F3FF04665F63707500000000003B
:1012B0000000000000F4FF04706F7274615F6469E5
:1012C00072736574000000010601706F7274615FD3
:1012D000646972636C72000000020601706F7274C0
:1012E000615F64697274676C000000030601706FCF
:1012F0007274615F64697200000000000000060102
:10130000706F7274615F6F757473657400000005AF
:101310000601706F7274615F6F7574636C720000A8
:1013200000060601706F7274615F6F757474676C8C
:10133000000000070601706F7274615F6F757400C2
:101340000000000000040601706F7274615F696E36
:1013500000000000000000080601706F7274625FF8
:10136000646972736574000000210601706F727405
:10137000625F646972636C72000000220601706F24
:101380007274625F64697274676C00000023060106
:10139000706F7274625F6469720000000000002068
:1013A0000601706F7274625F6F757473657400000C
:1013B00000250601706F7274625F6F7574636C72E2
:1013C000000000260601706F7274625F6F7574749E
:1013D000676C000000270601706F7274625F6F75A2
:1013E00074000000000000240601706F7274625FD8
:1013F000696E00000000000000280601706F727422
:10140000635F646972736574000000410601706F68
:101410007274635F646972636C720000004206015B
:10142000706F7274635F64697274676C000000436C
:101430000601706F7274635F6469720000000000DF
:1014400000400601706F7274635F6F75747365742A
:10145000000000450601706F7274635F6F757463FE
:101460006C72000000460601706F7274635F6F75E6
:101470007474676C000000470601706F7274635FDC
:101480006F7574000000000000440601706F7274F4
:10149000635F696E00000000000000480601706F85
:1014A0007274645F646972736574000000610601A0
:1014B000706F7274645F646972636C7200000062C2
:1014C0000601706F7274645F64697274676C000007
:1014D00000630601706F7274645F646972000000DB
:1014E000000000600601706F7274645F6F75747342
:1014F0006574000000650601706F7274645F6F753B
:1015000074636C72000000660601706F7274645F31
:101510006F757474676C000000670601706F7274F9
:10152000645F6F7574000000000000640601706F56
:101530007274645F696E00000000000000680601BC
:10154000706F7274655F6469727365740000008106
:101550000601706F7274655F646972636C7200007B
:1015600000820601706F7274655F64697274676CE3
:10157000000000830601706F7274655F6469720019
:101580000000000000800601706F7274655F6F7567
:1015900074736574000000850601706F7274655F76
:1015A0006F7574636C72000000860601706F727450
:1015B000655F6F757474676C000000870601706F5B
:1015C0007274655F6F75740000000000008406018E
:1015D000706F7274655F696E000000000000008823
:1015E0000601706F7274665F6469727365740000DF
:1015F00000A10601706F7274665F646972636C7239
:10160000000000A20601706F7274665F64697274F4
:10161000676C000000A30601706F7274665F6469F6
:1016200072000000000000A00601706F7274665F17
:101630006F7574736574000000A50601706F727495
:10164000665F6F7574636C72000000A60601706FB0
:101650007274665F6F757474676C000000A7060192
:10166000706F7274665F6F7574000000000000A4F4
:101670000601706F7274665F696E00000000000002
:1016800000A80601706F7274715F6469727365748B
:10169000000000C10701706F7274715F646972634A
:1016A0006C72000000C20701706F7274715F646930
:1016B0007274676C000000C30701706F7274715F11
:1016C000646972000000000000C00701706F72744E
:1016D000715F6F7574736574000000C50701706FEA
:1016E0007274715F6F7574636C72000000C60701DD
:1016F000706F7274715F6F757474676C000000C7EF
:101700000701706F7274715F6F75740000000000E4
:1017100000C40701706F7274715F696E0000000091
:10172000000000C80701706F7274725F64697273A1
:101730006574000000E10701706F7274725F646984
:1017400072636C72000000E20701706F7274725F66
:1017500064697274676C000000E30701706F727453
:10176000725F646972000000000000E00701706FA2
:101770007274725F6F7574736574000000E5070121
:10178000706F7274725F6F7574636C72000000E644
:101790000701706F7274725F6F757474676C00000C
:1017A00000E70701706F7274725F6F75740000005C
:1017B000000000E40701706F7274725F696E0000D0
:1017C0000000000000E80701757074696D65000095
:1017D00000000000000000FFFF0473797374696D5E
:1017E000650000000000000000FEFF040000000093
:1017F00000000000000000000000000000000A0DD2
:101800006F72202765652720746F206C6F616420DC
:1018100066726F6D20454550524F4D2E00556E6BD0
:101820006E6F776E20617267756D656E7420746F70
:10183000204C4F41443B207573652027666C3C6EFD
:101840003E2720746F206C6F61642066726F6D207C
:10185000464C41534800206461746120627974658C
:10186000732066726F6D20454550524F4D2E0020FB
:1018700070726F6772616D20627974657320616E3A
:101880006420004C6F6164656420005468697320B3
:1018900077696C6C206F76657277726974652074F5
:1018A00068652063757272656E742070726F6772FE
:1018B000616D20696E2052414D21202041726520CA
:1018C000796F7520737572653F20000A0D4E6F2089
:1018D00070726F6772616D20736176656420696EE6
:1018E00020454550524F4D21002E004E6F207375FC
:1018F000636820666C6173682066696C653B206D67
:10190000757374206265203020746F20002E0020D3
:10191000646174612062797465732066726F6D20F2
:10192000666C6173682066696C6520002070726F58
:101930006772616D20627974657320616E64200046
:101940004C6F616465642000546869732077696C2A
:101950006C206F7665727772697465207468652093
:1019600063757272656E742070726F6772616D213B
:10197000202041726520796F7520737572653F2054
:10198000000A0D4E6F2070726F6772616D20736177
:1019900076656420696E20666C6173682066696C88
:1019A0006520000A0D6F72202765652720746F205F
:1019B0007361766520746F20454550524F4D2E005F
:1019C000556E6B6E6F776E20617267756D656E74A4
:1019D00020746F20534156453B2075736520276660
:1019E0006C3C6E3E2720746F207361766520746FA7
:1019F00020464C415348004E6F2070726F677261F1
:101A00006D20696E2052414D3B206E6F7468696E87
:101A1000672073617665642E0020646174612062C2
:101A20007974657320746F20454550524F4D2E00D8
:101A30002070726F6772616D2062797465732061C6
:101A40006E642000536176656420005468697320D9
:101A500077696C6C206572617365207468652070AD
:101A6000726F6772616D206E6F7720696E204545D9
:101A700050524F4D21202041726520796F7520739F
:101A80007572653F2000206461746120627974651D
:101A90007320746F20666C6173682066696C6520C2
:101AA000002070726F6772616D20627974657320B7
:101AB000616E64200053617665642000212020411E
:101AC000726520796F7520737572653F20005468C8
:101AD00069732077696C6C20657261736520746826
:101AE000652070726F6772616D206E6F7720696E0E
:101AF00020666C6173682066696C652000206D61EA
:101B0000726B656420666F72206175746F737461A7
:101B100072742E0050726F6772616D20696E20665C
:101B20006C6173682066696C6520000A0D4E6F2039
:101B300070726F6772616D20736176656420696E83
:101B400020666C6173682066696C65200050726F56
:101B50006772616D20696E20454550524F4D206D72
:101B600061726B656420666F72206175746F737447
:101B70006172742E004E6F2070726F6772616D20FB
:101B8000736176656420746F20454550524F4D2136
:101B9000004175746F737461727420666C616720A4
:101BA00072656D6F7665642E000A0D4B4C42617351
:101BB000696320666F722041746D656C20415652D6
:101BC000204154786D65676131323861312076305B
:101BD0002E38000A0D53746F707065642061742094
:101BE0006C696E6520000A0D436F7265207772691B
:101BF0007474656E206279204B61726C204C756E36
:101C0000742C206261736564206F6E20476F72646C
:101C10006F6E20446F7567686D616E277320424157
:101C20005349433131000A0D4B4C426173696320C3
:101C3000636F72652076302E39000A0D524541449B
:101C400059003A20004552524F522023005E5E5EFA
:101C5000003A200020696E206C696E6520004552B4
:101C6000524F522023000A0D4E6F2070726F677220
:101C7000616D20696E206D656D6F72792E000A0DA1
:101C800050726F6772616D206572617365642E00BA
:101C90000A0D546869732077696C6C2065726173F2
:101CA00065207468652063757272656E7420707249
:101CB0006F6772616D21202041726520796F7520F8
:101CC000737572653F20004E6F2070726F6772618E
:101CD0006D206C6F6164656420696E206D656D6F49
:101CE00072792E0A0D006461746100270072656DBF
:101CF000004E6F207375636820666C6173682066A0
:101D0000696C652E00204E6F2070726F6772616D76
:101D10002E003A2000666C0020627974657320669C
:101D20007265650044796E616D6963206D656D6FE4
:101D3000727920706F6F6C202861727261797329DB
:101D40003A200020627974657320667265650056DA
:101D500061726961626C65206D656D6F72793A20A0
:101D60000020627974657320667265650050726F39
:101D70006772616D206D656D6F72793A2000556EE6
:101D80006B6E6F776E204155544F535420617267CC
:101D9000756D656E742E20204D75737420626520FC
:101DA0004F46462C2045452C20464C302C20464C96
:101DB000312C206F7220464C322E00496C6C6567C6
:101DC000616C206175746F73746172742076616CDC
:101DD000756520004175746F73746172742066724A
:101DE0006F6D20666C61736820004175746F737449
:101DF0006172742066726F6D20454550524F4D2EB2
:101E0000004175746F7374617274206E6F74206515
:101E10006E61626C65642E0011241FBECFEFDFE39C
:101E2000DEBFCDBF00E00CBF18BE19BE1ABE1BBE80
:101E300012E2A0E0B0E2E6E3FEE800E00BBF02C081
:101E400007900D92A631B107D9F71BBE16E3A6E1A4
:101E5000B2E201C01D92AA32B107E1F70E94FD1E55
:101E60000C9419470C94000024E030E420932134B2
:101E70003093223420937C3530937D3583ED97E485
:101E80008093D1349093D234F90101C011928091A2
:101E9000D1349091D2348E179F07C0F784ED97E428
:101EA0008093DC349093DD348093D4339093D53396
:101EB00083E596E88093CA349093CB3408959C01CF
:101EC0002C5F3F4BC9010895FC01DB0184E596E8D6
:101ED0008083918380ED97E08D939C93089520916A
:101EE0000040309101404091024050910340809168
:101EF000004090910140A0910240B091034028170A
:101F000039074A075B0741F02091004030910140BA
:101F10004091024050910340B901CA0108950895CB
:101F20008091A10985FFFCCF8DE08093A00980916D
:101F3000A10985FFFCCF8AE08093A0090895982F1E
:101F40008823C1F180911622882341F19636E1F071
:101F5000973638F4923681F0953651F09136A9F4DF
:101F60000DC0923779F0943729F09E3671F408C08D
:101F70009BE10BC099E009C098E007C097E005C05D
:101F80009AE003C09DE001C09CE01092162280916F
:101F9000A10985FFFCCF9093A00908959C3521F4F9
:101FA00081E08093162208958091A10985FFFCCFDE
:101FB0009093A0090895CF93DF93EC0102C00E9493
:101FC0009F0FFE01219684918823C9F7DF91CF915D
:101FD000089589EA9BE10E94DB0F0895CF93DF9378
:101FE000EC0102C00E949F0F89918823D9F7DF91ED
:101FF000CF910895982F8091A10985FFFCCF9093F0
:10200000A00908959091AB228091AC229817D1F34A
:10201000F894E091AC22F0E0E55DFD4D80812091E7
:10202000AC2230E02F5F3F4F2F7730702093AC22EF
:1020300078940895FF920F931F93CF93DF93EC0151
:1020400010E008E080E2F82E0E940210982F8D30F8
:10205000A9F488838091A10985FFFCCF8AE0809351
:10206000A0098091A10985FFFCCF8DE08093A00994
:10207000DF91CF911F910F91FF9008958830B9F4AF
:10208000112311F38091A10985FFFCCF0093A009D2
:102090008091A10985FFFCCFF092A0098091A10950
:1020A00085FFFCCF0093A00921971150CDCF8A3036
:1020B00059F28091A10985FFFCCF9093A0099993D3
:1020C0001F5FC2CF1F93142FFC01EE0FFF1F9F0154
:1020D00043E0220F331F4A95E1F7E20FF31FE15966
:1020E000FD4E44919C01220F331FF901A3E0EE0F36
:1020F000FF1FAA95E1F7E20FF31FE359FD4EA591EB
:10210000B491413011F41C931CC0423031F4812F42
:10211000952F8D939C93119714C0CD0140960497F1
:1021200080F4F894EA2FF0E0EF70F070EE0FFF1FEC
:10213000EE0FFF1FE55EFD4D1083518362837383B5
:1021400078941F910895FC01EE0FFF1F9F0143E05B
:10215000220F331F4A95E1F7E20FF31FE159FD4EBD
:1021600044919C01220F331FF90183E0EE0FFF1F02
:102170008A95E1F7E20FF31FE359FD4EA591B49163
:10218000413021F48C91282F30E005C0423031F4E9
:102190008D919C919C0140E050E052C0CD01409651
:1021A000049778F4EA2FF0E0EF70F070EE0FFF1F65
:1021B000EE0FFF1FE55EFD4D20813181428153818D
:1021C0003FC08FEFAF3FB80749F4209117223091FD
:1021D00018224091192250911A2232C08FEFAE3F3F
:1021E000B807F1F420910040309101404091024045
:1021F000509103408091004090910140A091024095
:10220000B0910340281739074A075B07C9F02091AE
:10221000004030910140409102405091034010C075
:10222000A45FBF4F29F020E030E040E050E008C05C
:102230002091C1223091C2224091C3225091C422E8
:10224000B901CA0108959C01220F331FF90173E0FF
:10225000EE0FFF1F7A95E1F7E20FF31FE359FD4EF2
:1022600065917491CB014096049750F4862F8F703E
:1022700090E0880F991F880F991F855E9D4D06C0BD
:102280008FEF6F3F780741F487E192E29C0144278A
:1022900037FD4095542F0CC08FEF643F780729F429
:1022A00020E030E040E050E003C09B0140E050E01F
:1022B000B901CA010895833028F020E030E040E001
:1022C00050E014C0E82FF0E0EE0FFF1FEE0FFF1FED
:1022D000EE5FFF4D808191819C0140E050E0FCE089
:1022E000220F331F441F551FFA95D1F7B901CA01B8
:1022F00008951F920F920FB60F9208B60F920BB669
:102300000F92112418BE1BBE8F939F93EF93FF93E0
:102310008091A009833021F481E08093D7340EC0EE
:10232000E091AB22F0E0E55DFD4D80838091AB2232
:1023300090E001968F7790708093AB22FF91EF91A0
:102340009F918F910F900BBE0F9008BE0F900FBE04
:102350000F901F9018951F920F920FB60F9208B60C
:102360000F9209B60F92112418BE19BE8F939F9336
:10237000AF93BF938091172290911822A0911922B8
:10238000B0911A220196A11DB11D8093172290933E
:102390001822A0931922B0931A2280911B229091A7
:1023A0001C22A0911D22B0911E220097A105B1050B
:1023B00059F00197A109B10980931B2290931C2227
:1023C000A0931D22B0931E2280911F229091202263
:1023D000A0912122B09122220097A105B10559F0C8
:1023E0000197A109B10980931F2290932022A09305
:1023F0002122B09322228091232290912422A09125
:102400002522B09126220097A105B10559F0019728
:10241000A109B1098093232290932422A09325221D
:10242000B09326228091272290912822A0912922E0
:10243000B0912A220097A105B10559F00197A10991
:10244000B1098093272290932822A0932922B09348
:102450002A22BF91AF919F918F910F9009BE0F904B
:1024600008BE0F900FBE0F901F9018951F920F92ED
:102470000FB60F9208B60F9209B60F92112418BE2C
:1024800019BE8F939F93AF93BF938091004090911B
:102490000140A0910240B09103400196A11DB11DE1
:1024A0008093004090930140A0930240B09303407A
:1024B000BF91AF919F918F910F9009BE0F9008BE71
:1024C0000F900FBE0F901F901895CF93DF93209120
:1024D000C00882E98093C0088091C008806480931E
:1024E000C008E0ECF7E094E0C0ECD8E035E0A0EC08
:1024F000B8E096833B838091C20887FFFCCF809130
:10250000C30813961C9213978091C20887FFFCCFD3
:102510008091C308958380FDECCF2093C008DF91A4
:10252000CF9108951F939B01AC011091C00882E9DF
:102530008093C0088091C00880648093C00884E0C4
:10254000E0ECF7E0868386E0E0ECF8E083838091BE
:10255000C20887FFFCCF8091C308E0ECF7E084E07D
:102560008583868380E2E0ECF8E083838091C20873
:1025700087FFFCCF8091C308CA01AA27BB27E0ECE4
:10258000F8E083838091C20887FFFCCF8091C30865
:10259000BB27A52F942F832FE0ECF8E08383809155
:1025A000C20887FFFCCF8091C308E0ECF8E02383EA
:1025B0008091C20887FFFCCF8091C30884E0E0ECE3
:1025C000F7E085830E9465121093C0081F9108955B
:1025D0006F927F928F929F92AF92BF92CF92DF9233
:1025E000EF92FF920F931F93CF93DF938B019C0188
:1025F000EA016090C00882E98093C0088091C00819
:1026000080648093C00884E0E0ECF7E0868386E095
:10261000E0ECF8E083838091C20887FFFCCF8091D3
:10262000C308E0ECF7E084E0858386838DEAE0EC84
:10263000F8E083838091C20887FFFCCF8091C308B4
:10264000C901AA27BB27E0ECF8E083838091C20888
:1026500087FFFCCF8091C308BB27A32F922F812F28
:10266000E0ECF8E083838091C20887FFFCCF809183
:10267000C308E0ECF8E003838091C20887FFFCCF39
:102680008091C3088881E0ECF8E083838091C208E0
:1026900087FFFCCF8091C3088981E0ECF8E0838359
:1026A0008091C20887FFFCCF8091C30884E0E0ECF2
:1026B000F7E085830E94651250ECA52E57E0B52EF9
:1026C00004E040EC842E48E0942E3DEA732E20EC8A
:1026D000C22E28E0D22EE12C90E1F92EEC0EFD1E48
:1026E000F5010683F40173828091C20887FFFCCF55
:1026F0008091C3088A81F60183838091C20887FF95
:10270000FCCF8091C3088B81F60183838091C2083E
:1027100087FFFCCF8091C30814E0F50105830E9478
:1027200065122296CE15DF05D9F6E0ECF7E01683A8
:10273000E0ECF8E013838091C20887FFFCCF809122
:10274000C308E0ECF7E084E08583868385E0E0EC75
:10275000F8E083838091C20887FFFCCF8091C30893
:10276000E0ECF8E013828091C20887FFFCCF8091F3
:10277000C30884E0E0ECF7E085836092C008DF9155
:10278000CF911F910F91FF90EF90DF90CF90BF906E
:10279000AF909F908F907F906F9008959B01AC01B8
:1027A0006091C00882E98093C0088091C00880646D
:1027B0008093C00884E0E0ECF7E0868383E0E0ECFF
:1027C000F8E083838091C20887FFFCCF8091C30823
:1027D000CA01AA27BB27E0ECF8E083838091C208F6
:1027E00087FFFCCF8091C308BB27A52F942F832F91
:1027F000E0ECF8E083838091C20887FFFCCF8091F2
:10280000C308E0ECF8E023838091C20887FFFCCF87
:102810008091C308E0ECF8E013828091C20887FF42
:10282000FCCF4091C308E0ECF8E013828091C2082D
:1028300087FFFCCF9091C30884E0E0ECF7E085834C
:102840006093C008392F20E0240F311DC90108957D
:102850009B01AC016091C00882E98093C00880911F
:10286000C00880648093C00884E0E0ECF7E08683D1
:1028700083E0E0ECF8E083838091C20887FFFCCF1F
:102880008091C308CA01AA27BB27E0ECF8E0838344
:102890008091C20887FFFCCF8091C308BB27A52F7A
:1028A000942F832FE0ECF8E083838091C20887FFA8
:1028B000FCCF8091C308E0ECF8E023838091C2084C
:1028C00087FFFCCF8091C308E0ECF8E01382809191
:1028D000C20887FFFCCF8091C30894E0E0ECF7E0EA
:1028E00095836093C0080895AF92BF92CF92DF9214
:1028F000EF92FF920F931F93CF93DF936C017A01B6
:102900008B015901C0E0D0E00DC0C801B7010E94A1
:102910002814F60181936F010894E11CF11C011D3C
:10292000111D2196CA15DB0580F3DF91CF911F9110
:102930000F91FF90EF90DF90CF90BF90AF900895F0
:10294000EF92FF920F931F937C010E94E346182F92
:1029500000E0C70101960E94E346080F111DC8015F
:102960001F910F91FF90EF900895CF92DF92EF9219
:10297000FF920F931F939B01AC01DC01CB010396E7
:10298000A11DB11D80509840A040B04040F088E2A9
:102990008093CC3420E030E040E050E015C0690185
:1029A000C9010E94A0147C0100E010E08701FF240F
:1029B000EE24C60102960E94A0149C0140E050E063
:1029C0002E0D3F1D401F511FB901CA011F910F91CC
:1029D000FF90EF90DF90CF900895AF92BF92CF928B
:1029E000DF92EF92FF920F931F931092AB221092FF
:1029F000AC221092D73460E070E080E090E00E945A
:102A0000B5147B018C016093C1227093C222809324
:102A1000C3229093C42264E070E080E090E00E94C2
:102A2000B5145B016C016093C5227093C62280933C
:102A3000C7229093C82268E070E080E090E00E9496
:102A4000B514AE0CBF1CC01ED11EA616B706C80614
:102A5000D906C1F080E098E4A8EEB1E08093C122ED
:102A60009093C222A093C322B093C42280E096E93F
:102A7000A0E0B0E08093C5229093C622A093C72225
:102A8000B093C82288E0809365068093610688E150
:102A90008093730680E38093A30924E0B22EB09262
:102AA000A40983E08093A509C090C122D090C222DE
:102AB000E090C322F090C4222091C5223091C6221A
:102AC0004091C7225091C82293E0220F331F441F28
:102AD000551F9A95D1F7C701B6010E946046215053
:102AE0001092A7092093A6098091A4098861809378
:102AF000A40900E418E0B0924008F80111821382A2
:102B000082E08783C701B60120E43FE140E050E066
:102B10000E946046F80126AB37ABB18610921B22AB
:102B200010921C2210921D2210921E2210921F221F
:102B300010922022109221221092222210922322FF
:102B400010922422109225221092262210922722DF
:102B5000109228221092292210922A2278941F91F2
:102B60000F91FF90EF90DF90CF90BF90AF900895BE
:102B70009B01AC01DC01CB010196A11DB11D805070
:102B80009840A040B04040F088E28093CC3420E0F0
:102B900030E040E050E006C0C9010E94A0149C0152
:102BA00040E050E0B901CA010895603028E07207A2
:102BB00020E0820720E0920740F088E28093CC3446
:102BC00020E030E040E050E007C0CB010E94E34647
:102BD000282F30E040E050E0B901CA01089588E1B3
:102BE00090E00E94E34608951F93CF93DF93EC019A
:102BF000162F0E94E346181721F0CE01612F0E9484
:102C0000F346DF91CF911F910895FF920F931F9389
:102C10008C01F62E672F0E94F415C80101966F2DC6
:102C20000E94F4151F910F91FF9008958F929F922B
:102C3000AF92BF92CF92DF92EF92FF920F931F93CA
:102C40006B017C0149015A01DC01CB010396A11DF6
:102C5000B11D80509840A040B04020F088E28093A1
:102C6000CC340CC0950144275527C601B9010E94F8
:102C70000516C6010296B4010E9405161F910F9118
:102C8000FF90EF90DF90CF90BF90AF909F908F908C
:102C900008950F931F938B019C01DC01CB010196DA
:102CA000A11DB11D80509840A040B04020F088E2A6
:102CB0008093CC3404C0C801BA010E9405161F914C
:102CC0000F910895603028E0720720E0820720E02D
:102CD000920720F088E28093CC340895CB01642FD2
:102CE0000E94F41508959B01BC01660F771FCB016C
:102CF00043E0880F991F4A95E1F7680F791F625AE0
:102D00007D4EC9010E94C14608956F927F928F92B5
:102D10009F92AF92BF92DF92EF92FF920F931F9319
:102D2000DF93CF93CDB7DEB72F97CDBFDEBF4C017A
:102D3000DD2463E1662E712C5E010894A11CB11C98
:102D40008D2D90E0869D7001879DF00C969DF00C76
:102D500011248701085C1D4EC8010E94C846892BBA
:102D6000D1F0C501B8010E94C146C5010E94D12819
:102D7000892B79F0F701E95BFD4E85919591A5913D
:102D8000B491F40180839183A283B38321E030E086
:102D900004C0D394D5CF20E030E0C9012F96CDBF39
:102DA000DEBFCF91DF911F910F91FF90EF90DF90E9
:102DB000BF90AF909F908F907F906F900895CF922B
:102DC000DF92EF92FF920F931F93DF93CF93CDB7D4
:102DD000DEB72F97CDBFDEBFFF2472E1E72E6E0175
:102DE0000894C11CD11CFE9C80011124025A1D4E66
:102DF000C8010E94C846892B59F0C601B8010E943B
:102E0000C146C6010E94D128892B89F4F394EBCFE7
:102E100020E030E0C9012F96CDBFDEBFCF91DF911A
:102E20001F910F91FF90EF90DF90CF900895E09168
:102E3000D834F091D93483E88193E093D834F09377
:102E4000D9348F2D90E00E94232821E030E0E2CF9A
:102E50002F923F924F925F926F927F928F929F92AA
:102E6000AF92BF92CF92DF92EF92FF920F931F9398
:102E7000DF93CF9300D00F92CDB7DEB78CE090E018
:102E80000E94A0148F5F9F4F19F48BEC98E1E1C072
:102E90002091DC343091DD348091D4339091D5335E
:102EA0002817390789F08BE898E10E94DB0F8DEA3B
:102EB00092E20E941A108091AD2290E00E94B146E9
:102EC0008937910509F0C7C08CE090E00E94A014FA
:102ED000F4EDCF2EF7E4DF2EC80ED91EC092DC34FD
:102EE000D092DD348EE090E00E94A0147601E80ECE
:102EF000F91EE092D433F092D53380E190E00E9445
:102F0000A0148C010C5F1F4B0093213410932234CA
:102F100082E190E00E94A014080F191F00937C35F5
:102F200010937D3586E190E00E94A0149C0140E062
:102F300050E029833A834B835C838C5A9947809372
:102F4000193490931A3427014C185D0800E010E002
:102F500009C0C8014A960E94E346D6018D936D01CF
:102F60000F5F1F4F04151505A0F3720100E010E07C
:102F70002AE130E040E050E0E20EF31E041F151F8E
:102F8000809021349090223480917C3590917D35D1
:102F9000881999095C01CC24B7FCC094DC2C662408
:102FA00077240EC0C7010E94E346D4018D934D01E2
:102FB0000894E11CF11C011D111D0894611C711C79
:102FC000C301A0E0B0E08A159B05AC05BD0550F338
:102FD00037014801E4E52E2EE6E83E2E0BC0C7017E
:102FE0000E94E346F10181931F010894E11CF11C4A
:102FF000011D111DC70186199709A0E0B0E02981C4
:103000003A814B815C8182179307A407B50738F397
:103010000E94DE3C80937E3590937F3583E898E173
:103020000E94DB0FB20180E090E00E94E5308FE665
:1030300098E10E94DB0F89819A81AB81BC81A80E47
:10304000B91ECA1EDB1EC601B5010E94E53086E529
:1030500098E10E94DB0F2496CDBFDEBFCF91DF91B8
:103060001F910F91FF90EF90DF90CF90BF90AF90A6
:103070009F908F907F906F905F904F903F902F9098
:103080000895CF93DF930E94DD27E091E134F09122
:10309000E234808190E0C0970A9718F0C0E0D0E059
:1030A00036C020E030E011C0C901B3E0880F991F9D
:1030B000BA95E1F7220F331F280F391F240F351F50
:1030C0003196E093E134F093E234E091E134F09111
:1030D000E2348081482F50E0405350404A3051053F
:1030E00018F3E9010E94DD27C330D10584F08BEE8F
:1030F00098E10E94DB0F62E070E080E090E00E94C7
:10310000E53089EE98E10E94DB0FCFEFDFEFCE01D3
:10311000DF91CF9108952F923F924F925F926F92DD
:103120007F928F929F92AF92BF92CF92DF92EF9257
:10313000FF920F931F93CF93DF931C01FC01EE0FBF
:10314000FF1FEE0FFF1FE050F04E2081922F92954F
:10315000907F80E06C01EE24FF246CE0862E912CA1
:10316000A12CB12C8C0C9D1CAE1CBF1CC501B40144
:103170000E94CE138F5F9F4F61F481E899E10E9416
:10318000DB0FB101882777FD8095982F0E94E530ED
:1031900057C12091DC343091DD348091D43390914B
:1031A000D5332817390789F088E499E10E94DB0FAD
:1031B0008DEA92E20E941A108091AD2290E00E9466
:1031C000B1468937910509F03BC1C501B4010E94A0
:1031D000CE138C010C52184B0093DC341093DD3469
:1031E0008EE090E0A0E0B0E0C80ED91EEA1EFB1E03
:1031F000C701B6010E94CE13080F191F0093D433E4
:103200001093D53382E090E0A0E0B0E0C80ED91E64
:10321000EA1EFB1EC701B6010E94CE138C010C5F93
:103220001F4B009321341093223482E090E0A0E001
:10323000B0E0C80ED91EEA1EFB1EC701B6010E94EF
:10324000CE13080F191F00937C3510937D3584E051
:1032500090E0A0E0B0E0C80ED91EEA1EFB1EC70138
:10326000B6010E94CE138C5A9947809319349093DB
:103270001A348090DC349090DD344090D4335090F8
:10328000D53348185908F101EE0FFF1FEE0FFF1F4D
:10329000EE5FFF4D808191815C01CC24DD248601AD
:1032A00075014CE0EE0CFF1C001F111F4A95D1F771
:1032B000C0E0D0E026C0C801B7010E942814D401A4
:1032C0008C930894E11CF11C011D111DD801C7014C
:1032D0009F70A070B0700097A105B10571F40894BB
:1032E000A11CB11CC11CD11C860175013CE0EE0C77
:1032F000FF1C001F111F3A95D1F70894811C911CE7
:103300002196C415D505B8F28090213490902234CE
:10331000C0917C35D0917D35C819D90966247724B0
:1033200028C0C801B7010E942814F40180830894C2
:10333000E11CF11C011D111DD801C7019F70A07077
:10334000B0700097A105B10571F40894A11CB11CDF
:10335000C11CD11C860175012CE0EE0CFF1C001F66
:10336000111F2A95D1F70894811C911C0894611CA7
:10337000711C6C167D06A8F294E5692E96E8792EEC
:103380008824992428C0C801B7010E942814D301B9
:103390008C930894E11CF11C011D111DD801C7017B
:1033A0009F70A070B0700097A105B10571F40894EA
:1033B000A11CB11CC11CD11C860175018CE0EE0C56
:1033C000FF1C001F111F8A95D1F70894611C711C06
:1033D0000894811C911C2091193430911A34C90130
:1033E000845596488816990670F2C455D648C20F7F
:1033F000D31F0E94DE3C80937E3590937F3580E41E
:1034000099E10E94DB0FB20180E090E00E94E5307C
:103410008CE299E10E94DB0FBE0180E090E00E9407
:10342000E5308FE099E10E94DB0FB101882777FD3D
:103430008095982F0E94E5308DE099E10E94DB0F86
:10344000DF91CF911F910F91FF90EF90DF90CF9080
:10345000BF90AF909F908F907F906F905F904F90B4
:103460003F902F9008950F931F93CF93DF930E9467
:10347000DD270091E1341091E234F80180818D3034
:1034800071F090E00E94B1468536910559F4F8013B
:10349000818190E00E94B14685369105F1F40E9449
:1034A000281723C086369105C1F4E8012196F8015A
:1034B000818190E00E94B1468C36910571F421968D
:1034C000C093E134D093E2340E944118FFEF8F3F64
:1034D0009F0759F00E948B1808C08DE198E10E9467
:1034E000DB0F8EEF97E10E94DB0FDF91CF911F91F1
:1034F0000F91089588E190E00E94E3468A3579F0C3
:103500008B3518F4853529F407C08B3559F08C3587
:1035100061F020E030E00FC00E9428170AC080E070
:1035200090E005C081E090E002C082E090E00E945F
:103530008B1821E030E0C9010895EF92FF920F93BC
:103540001F93CF93DF93EC018F3F910541F488E106
:1035500090E06FEF0E94F41581E99BE15BC0853537
:10356000910591F48CE090E00E94A0148F5F9F4F32
:1035700019F485E79BE14EC088E190E065E50E9483
:10358000F4158DE49BE146C08A35910511F410E0F5
:1035900009C08B35910511F411E004C08C359105FB
:1035A000D9F512E0E12FF0E0EE0FFF1FEE0FFF1F45
:1035B000E050F04E6081718180E090E0ECE0660FB9
:1035C000771F881F991FEA95D1F7645F7F4F8F4F50
:1035D0009F4F0E94CE13E12EFF2400E010E08F5F8A
:1035E0009F4F49F48BE29BE10E94DB0FC801B701BA
:1035F0000E94E53011C088E190E06C2F0E94F41524
:1036000084E19BE10E94DB0FC801B7010E94E53015
:103610008DEF9AE10E94DB0FDF91CF911F910F9107
:10362000FF90EF9008954F925F926F927F928F92EA
:103630009F92AF92BF92CF92DF92EF92FF920F9341
:103640001F93DF93CF93CDB7DEB76497CDBFDEBFB7
:103650008CE090E00E94A0148F5F9F4F81F08BE47C
:103660009AE10E94DB0FCE0101960E941A10898117
:1036700090E00E94B1468937910509F0F6C020918B
:10368000D4333091D5338091DC349091DD34281BD4
:10369000390B2A53364880917C3590917D35409185
:1036A000213450912234841B950B280F391F8091AF
:1036B000193490911A34820F931F875E974030F02F
:1036C00087E38093CC340E945931CFC088E190E0E9
:1036D0006FEF0E94F4158CE090E060E070E00E94D3
:1036E00005166091D4337091D5338091DC3490917C
:1036F000DD34681B790B8EE090E00E94051680E1B6
:1037000090E060E070E00E94051660917C35709159
:103710007D358091213490912234681B790B82E1B0
:1037200090E00E94051684E190E060E070E00E9465
:1037300005166091193470911A346455764886E103
:1037400090E00E940516E090DC34F090DD3440906B
:10375000D4335090D5334E185F0800E010E009C014
:10376000C8014A96F70161917F010E94F4150F5F2D
:103770001F4F04151505A0F35201CC24DD246090E1
:1037800021347090223480907C3590907D3586185D
:1037900097088AE190E0A0E0B0E0A80EB91ECA1E2A
:1037A000DB1E750186EE9FEFAFEFBFEFA80EB91ECF
:1037B000CA1EDB1E00E010E00BC0C701D3016D91F3
:1037C0003D010E94F4150F5F1F4F0894E11CF11C8E
:1037D0000815190590F3740100E010E0EA0CFB1CD9
:1037E0000C1D1D1D8AE190E0A0E0B0E0E80EF91E7E
:1037F0000A1F1B1F57016801B4E56B2EB6E87B2E2C
:103800000BC0C501D3016D913D010E94F4150894D0
:10381000A11CB11CC11CD11C4091193450911A3407
:1038200095012E193F09CA01845596482817390772
:1038300040F3E4E5F6E88E1A9F0A840E951E84E4B0
:103840009AE10E94DB0FB20180E090E00E94E53037
:1038500080E39AE10E94DB0FB40180E090E00E94D7
:10386000E53089E19AE10E94DB0F6496CDBFDEBFAF
:10387000CF91DF911F910F91FF90EF90DF90CF904C
:10388000BF90AF909F908F907F906F905F904F9080
:1038900008952F923F924F925F926F927F928F92F4
:1038A0009F92AF92BF92CF92DF92EF92FF920F93CF
:1038B0001F93CF93DF932091DC343091DD348091DE
:1038C000D4339091D5332817390719F487EF99E14C
:1038D0007FC20E94DD27C090E134D090E234F6012F
:1038E00080818D3079F090E00E94B1468536910557
:1038F00061F4F601818190E00E94B1468536910520
:1039000009F060C20E94131B65C28636910509F05A
:1039100059C2E6012196F601818190E00E94B146EC
:103920008C36910509F04EC22196C093E134D093B4
:10393000E2340E9441181C01FFEF8F3F9F0709F4FA
:1039400049C2FC01EE0FFF1FEE0FFF1FE050F04ECB
:10395000808191815C01CC24DD246CE0AA0CBB1C2D
:10396000CC1CDD1C6A95D1F7C601B501645F7F4FA1
:103970008F4F9F4F0E94CE138F5F9F4FE1F08EECD1
:103980009AE10E94DB0FB101882777FD8095982F7F
:103990000E94E5308CEB9AE10E94DB0F8DEA92E207
:1039A0000E941A108091AD2290E00E94B1468937A2
:1039B000910509F00FC2E091D433F091D5336091B5
:1039C000DC347091DD34EF01C61BD70BE0907C3501
:1039D000F0907D3500912134109122344701801AF6
:1039E000910A6090193470901A34230184E596E8A6
:1039F000481A590ACE01AA2797FDA095BA2F94011B
:103A0000442737FD4095542F820F931FA41FB51FE5
:103A10004A96A11DB11D9201442737FD4095542FB0
:103A2000820F931FA41FB51F81529E44A040B04037
:103A300030F087E38093CC340E945931CBC18FEFB3
:103A40008093E1221092D5221092D6228E2F861BCF
:103A50008093D722D093D8221092D9221092DA22C2
:103A60008E2D801B8093DB229092DC221092DD222F
:103A70001092DE2284E596E8E62DE81BE093DF2233
:103A8000852D992787FD9A958093E0229091C00813
:103A900082E98093C0088091C00880648093C00848
:103AA00084E0E0ECF7E0868386E0E0ECF8E08383F6
:103AB0008091C20887FFFCCF8091C308E0ECF7E05B
:103AC00084E08583868381E0E0ECF8E08383809165
:103AD000C20887FFFCCF8091C308E0ECF8E01382B6
:103AE0008091C20887FFFCCF8091C30884E0E0EC9E
:103AF000F7E085839093C008C601B5010E94921239
:103B0000C601B50149EC52E20E94E812F101EE0F44
:103B1000FF1FEE0FFF1FEE5FFF4D808191815C0163
:103B2000CC24DD24C0E0D0E040E050E029C0FA0120
:103B3000E753FD4DDE01AC52B84B8C9180834F5F53
:103B40005F4FF0E140305F07D1F4860175013CE042
:103B5000EE0CFF1C001F111F3A95D1F7C801B701E9
:103B60000E949212C801B70149EC52E20E94E81289
:103B70000894A11CB11CC11CD11C40E050E021964E
:103B80008091D4339091D5332091DC343091DD3461
:103B9000821B930BC817D90750F2C0E0D0E029C0B0
:103BA000FA01E753FD4DDE01AC5FBF4B8C91808382
:103BB0004F5F5F4F20E140305207D1F4860175011D
:103BC0002CE0EE0CFF1C001F111F2A95D1F7C80135
:103BD000B7010E949212C801B70149EC52E20E945B
:103BE000E8120894A11CB11CC11CD11C40E050E09B
:103BF000219680917C3590917D35209121343091B2
:103C00002234821B930BC817D90750F2C0E0D0E0D2
:103C100029C0FA01E753FD4DDE01AC5AB9478C913A
:103C200080834F5F5F4F80E140305807D1F48601B9
:103C300075019CE0EE0CFF1C001F111F9A95D1F737
:103C4000C801B7010E949212C801B70149EC52E2C3
:103C50000E94E8120894A11CB11CC11CD11C40E0B8
:103C600050E021968091193490911A3484559648E9
:103C7000C817D90770F2452B99F0860175018CE0C1
:103C8000EE0CFF1C001F111F8A95D1F7C801B70168
:103C90000E949212C801B70149EC52E20E94E81258
:103CA0009091C00882E98093C0088091C008806428
:103CB0008093C00884E0E0ECF7E0868386E0E0ECE7
:103CC000F8E083838091C20887FFFCCF8091C3080E
:103CD000E0ECF7E084E08583868381E0E0ECF8E0C7
:103CE00083838091C20887FFFCCF8091C3088CE159
:103CF000E0ECF8E083838091C20887FFFCCF8091DD
:103D0000C308E0ECF7E084E085839093C0088683E5
:103D100085E0E0ECF8E083838091C20887FFFCCF68
:103D20008091C308E0ECF8E013828091C20887FF1D
:103D3000FCCF8091C30884E0E0ECF7E0858385EB5D
:103D40009AE10E94DB0F6091D4337091D5332091BA
:103D5000DC343091DD34621B730B882777FD80954E
:103D6000982F0E94E53081EA9AE10E94DB0F2091B2
:103D70007C3530917D3524553648609119347091E9
:103D80001A34620F731F2091213430912234621B48
:103D9000730B882777FD8095982F0E94E53086E881
:103DA0009AE10E94DB0FB101882777FD8095982F5B
:103DB0000E94E5308091A10985FFFCCF8EE28093BF
:103DC000A00908C080EC99E10E94DB0F83EA99E129
:103DD0000E94DB0FDF91CF911F910F91FF90EF9029
:103DE000DF90CF90BF90AF909F908F907F906F901B
:103DF0005F904F903F902F900895809150008A607F
:103E0000809350008091510081FFFCCF88ED84BFEA
:103E100081E080934000809150008E7F809350001D
:103E20008091B4008C7FE0EBF0E084838BE0E0E4F1
:103E3000F0E0838387E080930004E0E0F4E0809189
:103E4000010480FDFACF80E290E082879387809121
:103E500002048360828310861186E0ECF7E084E040
:103E600085838183E0E4F6E080EB8583818380E4D1
:103E7000828382E98093C0088091C0088064809327
:103E8000C0080E94C54587E0E0EAF0E082837894AC
:103E90000E94522A81E090E00895E091D834F09198
:103EA000D9348081E80FF11DE093D834F093D934F0
:103EB0000895E091D834F091D9348081E80FF11D54
:103EC000E093D834F093D9340895A091D834B091C8
:103ED000D934FD012191E093D834F093D9342439B9
:103EE00051F411962D913C9112971396A093D834CA
:103EF000B093D93418C0223819F420E030E015C04E
:103F000011968D919C911297FD013396233831F4CF
:103F10009C01E093D834F093D93407C0E093D834AF
:103F2000F093D9349C01215F3F4FC9010895E0917E
:103F3000B334EE2321F48DE18093CC340895E15025
:103F4000E093B334F0E0EE0FFF1FEA5FF94C80819D
:103F500091818093D8349093D93408950895089529
:103F6000CF93DF93E091E034EE2331F48FE180933F
:103F7000CC340E94593124C0C091D834D091D93466
:103F8000F0E0EE0FFF1FE852FC4C8081918180939E
:103F9000D8349093D9340E94AC428AE695E368E322
:103FA0000E949D27611571058105910549F4C09313
:103FB000D834D093D9348091E03481508093E03468
:103FC000DF91CF910895CF93DF930E943136C09156
:103FD000D834D091D93480912034882351F0809105
:103FE000D4339091D53301978093D8349093D934BA
:103FF00006C02396C093D834D093D93423970E9417
:1040000031362091B334203121F48CE18093CC34CB
:1040100013C0E22FF0E0EE0FFF1FEA5FF94C809132
:10402000D8349091D934808391832F5F2093B33417
:10403000C093D834D093D934DF91CF9108950E94A2
:10404000900F81E08093C9341092E3341092E434ED
:104050008091D4339091D53301978093D834909345
:10406000D9340895CF93DF932091E034203131F497
:104070008EE18093CC340E94593141C0E22FF0E0B0
:10408000EE0FFF1FE652FC4C8091D8349091D9344A
:10409000808391832F5F2093E034C1E0D0E0E091F2
:1040A000D833F091D933E093D834F093D9343097A2
:1040B00031F18091D4339091D533E817F90719F491
:1040C0000E941F201CC082819F01280F311D209358
:1040D000D8333093D9333396E093D834F093D9342E
:1040E0000E943136E091D834F091D934E081E93141
:1040F00011F42196D4CFEA3191F6219781F6DF9120
:10410000CF91089583ED9BE10E94DB0F6091E33432
:104110007091E43480E090E00E94E5301092C93460
:104120008091D8339091D93380938435909385359D
:104130001092E3341092E4348091D4339091D533CB
:1041400001978093D8349093D93408950E943136E2
:10415000E091D834F091D934218132813396E093C3
:10416000D834F093D93450912034552341F08091C4
:10417000D4339091D5338093D8339093D933E09151
:10418000D833F091D9336091D4337091D533E61799
:10419000F70721F4E091DC34F091DD3480819181E6
:1041A0002817390720F4E091DC34F091DD34808168
:1041B000918182179307B1F4E093D834F093D93406
:1041C000552341F01092203481E08093B0340E9456
:1041D0000F3808953396E093D834F093D9340E9481
:1041E0003136089542812817390728F0E40FF11D70
:1041F000E617F707E1F68BE18093CC340895AF9290
:10420000BF92CF92DF92EF92FF920F931F93CF93C3
:10421000DF93E091D834F091D9341081103731F028
:10422000133721F0143711F000E00DC03196E09300
:10423000D834F093D9340E943136E091D834F091DB
:10424000D934012F10810E94651F7C01143919F0A7
:10425000C0E0D0E034C08091D8349091D934019638
:104260008093D8349093D9340E94AC428091D83452
:104270009091D93401968093D8349093D934809119
:10428000CC34882309F082C0C7010E945F0FFC0173
:10429000C081D1818AE695E368E30E949D278881E9
:1042A00099816817790720F089E18093CC346EC03A
:1042B0002296660F771F660F771FC60FD71F0E94C3
:1042C00031368091D8349091D93401968093D83486
:1042D0009093D9340E94AC428091CC34882309F069
:1042E00055C08AE695E368E30E949D275B016C0157
:1042F000133831F4C701B601A5010E94621046C00F
:10430000143929F4688379838A839B833FC0C7016A
:104310000E945F0FFC010023D9F02081318142818E
:104320005381003749F4CA01AA27BB27F9010BB60C
:104330008BBFA0820BBE2AC0043779F4CA01AA271A
:10434000BB27F9010BB68BBFA192B0820BBE1EC07A
:104350009C01442737FD4095542FCA01AA27BB274B
:10436000F9010BB68BBFA192B0820BBE2E5F3F4FFF
:104370004F4F5F4F7A0100271127C601AA27BB279D
:10438000F9010BB6EBBE819390830BBEDF91CF9109
:104390001F910F91FF90EF90DF90CF90BF90AF9063
:1043A00008958FEF8093CD3308951092CD33089503
:1043B00008958091D8349091D93403968093D8345D
:1043C0009093D9340E94AC428091D8349091D934E2
:1043D00001968093D8349093D93408951F93182F61
:1043E00082958F708A3008F0895F805D0E94FA0F95
:1043F000812F8F708A3008F0895F805D0E94FA0FEC
:104400001F910895EF92FF920F931F930E94D9215D
:104410008AE695E368E30E949D277B018C01892F42
:104420009927AA27BB270E94EE21C801AA27BB27EC
:104430000E94EE21BB27A12F902F8F2D0E94EE21ED
:104440008E2D0E94EE211F910F91FF90EF90089505
:10445000EF92FF920F931F930E94D9218AE695E372
:1044600068E30E949D277B018C01BB27A92F982F11
:10447000872F0E94EE218E2D0E94EE211F910F9119
:10448000FF90EF9008950E94D9218AE695E368E3B2
:104490000E949D27862F0E94EE2108950E94D92117
:1044A0008AE695E368E30E949D27862F0E94FA0F13
:1044B00008950E94D9218AE695E368E30E949D272A
:1044C00089E00E94FA0F0895EF92FF920F931F93D5
:1044D0000E943136E091D834F091D934E08110E077
:1044E0007BC0EB37B1F1EC3720F4E63309F05FC065
:1044F0003BC0EC3759F1E23A09F059C0E091D834A9
:10450000F091D9346181E62EFF2400E010E08EEFB7
:104510009FEFAFEFBFEFE80EF91E0A1F1B1F339688
:10452000E093D834F093D934CF01B7010E94AE257F
:10453000B7016F5F7F4F8091D8349091D934860F47
:10454000971F8093D8349093D93423C089E00E9478
:10455000FA0F8091D8349091D93401968093D83451
:104560009093D93411E031C0E091D834F091D9342E
:1045700081818B3099F08C3028F4823061F0873063
:10458000B1F405C08D3069F08E3089F40DC00E9401
:10459000592210E01AC00E944E2228C00E94022216
:1045A00025C00E94432222C00E9428221FC00E94D0
:1045B000AC428091CC348823E9F48AE695E368E341
:1045C0000E949D270E94E53011C00E943136E09183
:1045D000D834F091D934E081ED3719F0EA3709F099
:1045E00080CF112339F40E94900F04C080E20E9412
:1045F000FA0FCFCF1F910F91FF90EF900895EF9298
:10460000FF920F931F93CF93DF93E0901934F090B4
:104610001A340E943136E091D834F091D934808137
:1046200084FD02C081E22FC0818192810F960E9499
:104630005F0FEC018091D8349091D9340496809327
:10464000D8349093D9340E94AC428091D834909160
:10465000D93401968093D8349093D9348881998144
:10466000AA81BB810097A105B10509F047C000915F
:10467000193410911A348AE695E368E30E949D2765
:1046800077FF04C087E28093CC3447C0409119344F
:1046900050911A34088319831A821B826F5F7F4FEF
:1046A000F801608371834E5F5F4FCB01880F991FC4
:1046B000880F991F840F951F4250504080931934E2
:1046C00090931A342091783530917935281739072D
:1046D00020F0FA0180E090E00EC089E08093CC34B5
:1046E000E0921934F0921A3418C0128213821482A4
:1046F00015820196349686179707B8F30E943136D3
:10470000E091D834F091D93480818D3731F03196F1
:10471000E093D834F093D93478CFDF91CF911F91C3
:104720000F91FF90EF9008950895089508950895CA
:10473000089508950895089508950895089580911D
:104740002034882329F083E38093CC340E945931AC
:104750000895CF93DF93C091D834D091D93480910C
:10476000DC349091DD348093D8349093D9348093A5
:10477000C0349093C134E091D834F091D93482811F
:104780009F01280F311D2093C0343093C1343396DC
:10479000E093D834F093D9340E943136E091D83484
:1047A000F091D93480818C3051F43296E093C0344A
:1047B000F093C134C093D834D093D9341AC0209127
:1047C000C0343091C1348091D4339091D5332817BF
:1047D000390751F4C093D834D093D93486E280930A
:1047E000CC340E94593105C02093D8343093D93449
:1047F000C2CFDF91CF910895CF93DF93C091D8348A
:10480000D091D9348091C0349091C1348093D83400
:104810009093D9348091D8349091D9340396809371
:10482000D8349093D9340E943136E091D834F09145
:10483000D93480818C3051F43396E093C034F093B6
:10484000C134C093D834D093D9341BC0E091C03464
:10485000F091C1348091D4339091D533E817F907A2
:1048600041F4C093D834D093D93486E28093CC34C9
:1048700008C08281E80FF11DE093C034F093C13489
:10488000C9CFDF91CF910895CF92DF92EF92FF923F
:104890000F931F930E9431360E94651F8C010E9466
:1048A0000210C82EC8010E945F0FFC01DD24EE2417
:1048B000FF24C082D182E282F3821F910F91FF9088
:1048C000EF90DF90CF900895CF93DF930E94313621
:1048D0000E94651F9C019091CE338EE0989FE0016D
:1048E0001124CB5EDB4C888199812817390731F080
:1048F00084E28093CC340E94593145C0C9010E94A2
:104900005F0FFC0120813181428153818A819B812B
:10491000AC81BD81280F391F4A1F5B1F2083318363
:10492000428353838A819B81AC81BD81B7FF0AC0DA
:104930008E819F81A885B985281739074A075B07AB
:10494000B4F40DC00097A105B10589F08E819F8157
:10495000A885B98582179307A407B50744F4809109
:10496000CE3381508093CE330E9431360CC08A857D
:104970009B858093D8349093D9348C859D85809382
:10498000E3349093E434DF91CF910895DF92EF9276
:10499000FF920F931F93D82E8091D8349091D934E1
:1049A00001968093D8349093D9340E9431360E9476
:1049B000AC420E9431368091D8349091D93401961E
:1049C0008093D8349093D9340E9431368091D83472
:1049D0009091D93401968093D8349093D9340E9421
:1049E000AC428AE695E368E30E949D277B018C0137
:1049F0008AE695E368E30E949D2722E0D216A1F0A3
:104A000034E0D316F9F041E0D41611F580E090E0DF
:104A10002FEF30E040E050E0E222F32204231523A0
:104A20004E2D0E94621614C080E090E02FEF3FEF01
:104A300040E050E0E222F32204231523A7010E9464
:104A4000491606C080E090E0A80197010E94161662
:104A50001F910F91FF90EF90DF90089584E00E94E6
:104A6000C624089582E00E94C624089581E00E9431
:104A7000C62408950E94AC420E9431368091D834F9
:104A80009091D93401968093D8349093D9340E9470
:104A900031368AE695E368E30E949D279B01AC01CD
:104AA0008091CC348823C1F5E091D834F091D93489
:104AB000232B31F08081883A79F50E94A620089551
:104AC0008081883A79F43396E093D834F093D934DE
:104AD0000E943136E091D834F091D9348081893305
:104AE000D9F40AC08091D8339091D933019780933B
:104AF000D8349093D93408953196E093D834F09314
:104B0000D9340E943136E091D834F091D934808183
:104B1000883A11F40E94A62008951F93E091E13491
:104B2000F091E23480818D3211F010E006C03196B0
:104B3000E093E134F093E23411E00E94112E9B01E6
:104B4000AC01112339F050954095309521953F4F98
:104B50004F4F5F4FB901CA011F9108950F931F93E3
:104B6000CF93DF938C01EB0106C0F80181918F0197
:104B70000E949F0F21972097C1F7DF91CF911F913E
:104B80000F910895EF92FF920F931F93E091E134FC
:104B9000F091E2348081843241F43196E093E13443
:104BA000F093E2340E94B52E02C00E948D257B0155
:104BB0008C010E94DD27E091E134F091E2348081A4
:104BC0008D3071F08C3231F43196E093E134F09312
:104BD000E23406C085E18093CC340E94593109C08B
:104BE0000E94651F0E945F0FFC01E082F182028338
:104BF00013831F910F91FF90EF9008950E94DD277E
:104C0000E091E134F091E23480818D30C9F00E946E
:104C1000C2258091CC34882399F40E943136E091EA
:104C2000D834F091D93480818D3769F08A3759F0C2
:104C30003196E093D834F093D9340E943136DECFE8
:104C400021E030E002C020E030E0C9010895809109
:104C5000C0349091C134892B21F40E94A9230E9471
:104C6000FC238091C0349091C1348093E1349093BF
:104C7000E2340E9431360E94FE252091E1343091C9
:104C8000E234019769F42E5F3F4F2093C034309394
:104C9000C1340E94FC238091CC34882311F304C0DA
:104CA0002093C0343093C1340895EF92FF920F9354
:104CB0001F930E943136E091D834F091D93480812D
:104CC000823A01F5018110E00250104083E0E82EA5
:104CD000F12CEE0EFF1EC701B8010E94AE250F5F3A
:104CE0001F4FE00EF11EE092D834F092D9340E94AA
:104CF00031368091D8349091D93401968093D8344C
:104D00009093D9340E9431368FE30E94FA0F80E2EB
:104D10000E94FA0F0E943D2A0E94900F0E9479364D
:104D2000882321F40E94FE25892B71F710922636E4
:104D30001F910F91FF90EF9008950F931F93809113
:104D4000CE338A3031F483E28093CC340E945931DF
:104D5000B8C00E9431360091D8341091D9340E94E5
:104D6000651F4091CE33242F30E0220F331FF9010D
:104D700073E0EE0FFF1F7A95E1F7E21BF30BED5D99
:104D8000FB4C80839183842F90E0880F991FFC0156
:104D900053E0EE0FFF1F5A95E1F7E81BF90BED5DAD
:104DA000FB4C8091E3349091E434848795870093A1
:104DB000D8341093D9340E94FF200E94313680915C
:104DC000D8349091D93401968093D8349093D934C3
:104DD0000E9431360E94AC421091CE338AE695E3B0
:104DE00068E30E949D27212F30E0220F331FF90135
:104DF00003E0EE0FFF1F0A95E1F7E21BF30BED5DF9
:104E0000FB4C66837783808791878091CE3390E0D7
:104E1000FC0113E0EE0FFF1F1A95E1F7E81BF90BF9
:104E2000EE0FFF1FEB5DFB4C81E090E0A0E0B0E0F7
:104E300080839183A283B3830E943136E091D8347A
:104E4000F091D93480818A3319F53196E093D834C2
:104E5000F093D9340E9431360E94AC420091CE3397
:104E600010E08AE695E368E30E949D27F801A3E03D
:104E7000EE0FFF1FAA95E1F7E01BF10BEE0FFF1FEE
:104E8000EB5DFB4C60837183828393830E94313698
:104E90002091CE33822F90E0880F991FFC0133E0E0
:104EA000EE0FFF1F3A95E1F7E81BF90BED5DFB4CA8
:104EB0008091D8349091D934828793872F5F209343
:104EC000CE331F910F910895FC01118240836283BC
:104ED00073830895FC011182408362837383089574
:104EE000FC018181882331F46093CC340E945931D4
:104EF00080E00895815081830280F381E02DE80FE6
:104F0000F11D80810895DC0111969C9111978C917F
:104F1000981729F44093CC340E9459310895129681
:104F2000ED91FC911397E90FF11D608311968C911F
:104F300011978F5F11968C930895FC0181818823CE
:104F400049F46093CC340E94593120E030E040E0D5
:104F500050E010C08150818390E0880F991F880F26
:104F6000991F0280F381E02DE80FF91F2081318124
:104F700042815381B901CA010895DC0111963C9127
:104F800011978C91381729F42093CC340E94593111
:104F90000895832F90E0880F991F880F991F12960C
:104FA000ED91FC911397E80FF91F408351836283C1
:104FB00073833F5F11963C93089505C03196E0934B
:104FC000E134F093E234E091E134F091E234808115
:104FD0008032A1F30895E091E134F091E2348081D0
:104FE00090E0C0970A97E8F019C0CA01B3E0880FB3
:104FF000991FBA95E1F7440F551F480F591F460FE7
:10500000571F3196E093E134F093E234421753078F
:1050100010F09A010AC081E08093CC3440E050E067
:1050200010C040E050E020E030E0E091E134F09149
:10503000E2348081682F70E0605370406A307105FF
:10504000A0F2CA010895E091D834F091D934819347
:105050009193E093D834F093D9340895E091D83403
:10506000F091D9348083918312823396E093D834BF
:10507000F093D934089590E006C03196E093E1347E
:10508000F093E2349F5FE091E134F091E23480816B
:10509000803299F39923C1F0A091D834B091D934DA
:1050A000923058F0FD018FE7819311969C933196D1
:1050B000E093D834F093D9340895FD018EE78193BD
:1050C000E093D834F093D9340895E091E134F0912D
:1050D000E234808108958091E1349091E234019628
:1050E0008093E1349093E2340895E091D834F091C4
:1050F000D9346193719381939193E093D834F09371
:10510000D9340895282FE091D834F091D934809182
:10511000B6349091B73480589F4FE817F90721F4BF
:1051200084E18093CC34089520838091D834909189
:10513000D93401968093D8349093D9340895AF929E
:10514000BF92CF92DF92FF920F931F93CF93DF9383
:105150005C016B01C0E0D0E013C0F501EC0FFD1F56
:10516000808190E00E94B9468C018F2D90E00E94D2
:10517000B9460817190719F0C0E0D0E007C021961A
:10518000F601EC0FFD1FF080FF2039F7CE01DF9113
:10519000CF911F910F91FF90DF90CF90BF90AF9074
:1051A00008950F931F93182F092F8091E134909148
:1051B000E234612F702F0E949F28892B19F4A0E000
:1051C000B0E013C0E12FF02FDF010D900020E9F7D0
:1051D0001197AE1BBF0B8091E1349091E2348A0F9E
:1051E0009B1F8093E1349093E234CD011F910F9186
:1051F000089515C110921B340E943B288CE090E268
:105200000E94D128892B19F00E948D2BF2C081E1D8
:1052100090E20E94D128892B19F00E94802DE9C0CC
:1052200085E190E20E94D128892B19F00E94683212
:10523000E0C08AE190E20E94D128892B19F00E94F7
:10524000C430D7C082E290E20E94D128892B19F0A5
:105250000E94AD2DCEC088E290E20E94D128892B19
:1052600019F00E94A92DC5C08DE290E20E94D128BC
:10527000892B19F00E94C933BCC080E390E20E94E0
:10528000D128892B19F00E94252BB3C087E390E227
:105290000E94D128892B19F00E943333AAC08AE3D7
:1052A00090E20E94D128892B19F00E948932A1C076
:1052B00080E490E20E94D128892B19F00E941B32D1
:1052C00098C086E490E20E94D128892B19F00E94B0
:1052D000C3328FC08AE490E20E94D128892B19F052
:1052E0000E94753286C08FE490E20E94D128892BFB
:1052F00019F00E94302B7DC084E590E20E94D128F5
:10530000892B19F00E94CF3074C08AE590E20E9488
:10531000D128892B19F00E943B2B6BC08EE590E2BF
:105320000E94D128892B19F00E94952B62C082E639
:1053300090E20E94D128892B19F00E94563259C060
:1053400086E690E20E94D128892B19F00E94462B14
:1053500050C08BE690E20E94D128892B19F00E9460
:10536000512B47C081E790E20E94D128892B19F088
:105370000E94B7313EC087E790E20E94D128892B76
:1053800019F00E94383535C08DE790E20E94D1288F
:10539000892B19F00E9434352CC083E890E20E94DA
:1053A000D128892B19F00E943C3523C087E890E270
:1053B0000E94D128892B19F00E941F321AC08EE852
:1053C00090E20E94D128892B19F00E94173211C057
:1053D00080E990E20E94D128892B19F00E94912B3C
:1053E00008C082E990E20E94D128892B91F50E94A1
:1053F0007C2D8091CC34882361F50E943B28E0917C
:10540000E134F091E234E081EA3319F40E94112B87
:1054100006C0ED3021F082E08093CC340895E09115
:10542000E134F091E23480818D3009F0E3CEE091F7
:10543000D834F091D9348DE780838091203488234B
:1054400041F42091D83486E895E3281B2F5F209300
:10545000883508951F93182F90E00E949F46892B4E
:1054600039F420E030E0812F90E0C0970A9710F4E3
:1054700021E030E0C9011F9108950F931F9306EEBC
:1054800014E3C8010E941A10F80101900020E9F706
:1054900031978DE080830093E1341093E2341F91C3
:1054A0000F910895DF92EF92FF920F931F93DF9376
:1054B000CF930F920F92CDB7DEB70E94ED140E94EA
:1054C000B23C0E949D3C89E194E3BE016F5F7F4F37
:1054D0000E94640F8091193490911A3429813A8185
:1054E000820F931F80937835909379350E947A1AB2
:1054F000892B11F00E9487380E94900F0E94900F14
:105500000E94E90F86E29CE10E94DB0F86EE9BE1A0
:105510000E94DB0F81E08093203416E8E12E15E332
:10552000F12EDD24D39480912034882321F08AE366
:105530009CE10E94DB0F109220341092CC34109228
:10554000B0340E94900F8EE30E94FA0F0E943D2A11
:1055500005C03196E093E134F093E234E091E13418
:10556000F091E23480818032A1F386E695E36BEF1F
:1055700073E34EE10E946A278AE695E36DED72E3DC
:105580004CE30E9464270E947F3B892B61F60091C7
:105590007C3510917D35E092D834F092D934109258
:1055A000FA330E94EB279C010097D1F0E091E1349F
:1055B000F091E23480818D3021F4C9010E94F93CE0
:1055C00024C010922034E091D834F091D934208353
:1055D000318312823396E093D834F093D93402C0E9
:1055E000D09220348091CC34882379F40E94F92819
:1055F0008091CC34882349F480912034882319F099
:105600000E94473602C00E94DD3D8091CC34882341
:1056100009F489CF0E94593100937C3510937D3570
:1056200082CFE091D834F091D9348AE78193E09326
:10563000D834F093D9348091E1349091E2340196DA
:105640008093E1349093E2340895E091D834F0915E
:10565000D93484E18193E093D834F093D934089518
:10566000E091D834F091D93487E18193E093D83434
:10567000F093D9340895E091D834F091D93488E189
:105680008193E093D834F093D9340895E091D834DD
:10569000F091D93486E08193E093D834F093D934F3
:1056A0000895E091D834F091D93487E08193E09364
:1056B000D834F093D9340895A091D834B091D93426
:1056C000FD01819311961C9211973196E093D83485
:1056D000F093D93422E0E091E134F091E234819109
:1056E000E093E134F093E234E091D834F091D9348E
:1056F0008193E093D834F093D9348D3011F02F5F3B
:10570000EACF8091E1349091E23401978093E134C3
:105710009093E23411962C9308958CE00E945C2BB8
:10572000089584E40E945C2B08958AE00E945C2B1B
:10573000089587E990E20E94D128892B11F082E335
:1057400008958AE990E20E94D128892B11F083E321
:1057500008958DE990E20E94D128892B11F085E30C
:10576000089580EA90E20E94D128892B11F080E30D
:10577000089582EA90E20E94D128892B11F081E3FA
:10578000089584EA90E20E94D128892B11F480E0E8
:10579000089584E3089586EA90E20E94D128892B37
:1057A00011F080E208958AEA90E20E94D128892BC4
:1057B00011F081E208958DEA90E20E94D128892BB0
:1057C00011F480E0089582E2089581EB90E20E9456
:1057D000D128892B11F080E4089583EB90E20E9498
:1057E000D128892B11F081E4089585EB90E20E9485
:1057F000D128892B11F080E5089587EB90E20E9473
:10580000D128892B11F081E5089589EB90E20E945F
:10581000D128892B11F082E508958DEB90E20E944A
:10582000D128892B11F480E0089580E608959F9295
:10583000AF92BF92CF92DF92EF92FF920F931F939E
:10584000182F00E061E7962E50E7B52E43E7A42E0F
:1058500034E7D32E22E7C22E90E1E92E81E1F82E23
:105860000E943B2883EB90E20E94D128892B31F0E3
:10587000E091D834F091D934C1922FC08FEB90E2EF
:105880000E94D128892B31F0E091D834F091D9349D
:10589000D19223C083EC90E20E94D128892B31F071
:1058A000E091D834F091D934A19217C087EC90E2FE
:1058B0000E94D128892B31F0E091D834F091D9346D
:1058C000B1920BC089EC90E20E94D128892B49F05B
:1058D000E091D834F091D9349192E093D834F09398
:1058E000D9340E943B28E091E134F091E234808188
:1058F0008832B9F5E091D834F091D934E192E0934F
:10590000D834F093D9348091E1349091E234019607
:105910008093E1349093E234812F0E94172C809180
:10592000CC34882309F077C0E091E134F091E2347F
:105930008081893211F084E060C0E091D834F09128
:10594000D934F192E093D834F093D9348091E13492
:105950009091E23401968093E1349093E23411E027
:105960001EC00E941D2F982F882369F40E94403585
:10597000982F882341F40E94DF16982F882319F46A
:105980000E94FA2F982F8091CC34882309F043C0CD
:10599000112321F0911711F085E02FC0192F0E94DB
:1059A0003B28E091E134F091E234E081ED3099F16F
:1059B000EA3389F1EC3279F1EB3369F1E93259F1EB
:1059C0001130C1F40E94E52B8823D9F40E94CB2B1F
:1059D0008823B9F480911B34882339F00023D9F44B
:1059E0000E94992B882361F407C080912736882371
:1059F00019F011C083E101C086E08093CC340BC064
:105A000001E0E091D834F091D9348193E093D83417
:105A1000F093D93425CF1F910F91FF90EF90DF9035
:105A2000CF90BF90AF909F9008951F930E94DF1674
:105A3000182F882329F40E94FA2F182F882311F198
:105A40008091CC348823F1F40E943B28E091E1342A
:105A5000F091E2348191E093E134F093E2348D33BC
:105A600021F083E08093CC340DC0E091D834F091E4
:105A7000D93489E78193E093D834F093D934812FD6
:105A80000E94172C1F910895E091D834F091D934D9
:105A90008193E093D834F093D9340E943B2883EC6F
:105AA00090E20E94D128892B31F0E091D834F09116
:105AB000D93483E717C08FEB90E20E94D128892B5D
:105AC00031F0E091D834F091D93484E70BC087EC01
:105AD00090E20E94D128892B51F0E091D834F091C6
:105AE000D93480E78193E093D834F093D9340E947D
:105AF0003B280E94152D089582E00E94442D0895B0
:105B000081E00E94442D0895E091D834F091D93479
:105B10008193E093D834F093D9340E943B28E091EC
:105B2000D834F091D93488EA8193E093D834F09353
:105B3000D9340E94EB279C01009719F482E18093ED
:105B4000CC348091CC34882319F4C9010E942328D5
:105B5000089582E10E94842D08958FE00E94842D93
:105B60000895E091E134F091E2348081883219F4B3
:105B700024E930E002C020E030E0C9010895282F78
:105B8000DB0140917C3550917D35FA018193E093A2
:105B90007C35F0937D3590E08C91E0917C35F091EF
:105BA0007D358193E0937C35F0937D358C91811127
:105BB00011969F5F9E3081F7243851F0243941F0CF
:105BC000223811F494E005C0213811F088E01BC0A0
:105BD00095E081E020917C3530917D35F90111927D
:105BE000E0937C35F0937D358F5F981798F720937D
:105BF0007C3530937D358091D1349091D2348217A9
:105C0000930730F489E08093CC34EFEFFFEF07C0C7
:105C10008091213490912234FA01E81BF90BCF01D5
:105C200008950F931F93CF93DF93E091E134F091A8
:105C3000E234808190E0C0970A9728F420E030E0B9
:105C400040E050E025C082E016C0CA01B9012AE058
:105C500030E040E050E00E9421469B01AC01CE01C3
:105C6000AA2797FDA095BA2F280F391F4A1F5B1F3F
:105C700057FF08C08AE08093CC3420E030E040E059
:105C800050E012C00F5F1F4F0093E1341093E234D5
:105C90000091E1341091E234F8018081C82FD0E006
:105CA000E097CA30D10588F2B901CA01DF91CF91DE
:105CB0001F910F910895CF93DF93C091D834D09165
:105CC000D934DE0182EA8D93CD0101968093D834D8
:105CD0009093D934E091E134F091E234219111961E
:105CE0002C9301968093D8349093D934E093E13487
:105CF000F093E23422E018C08D3019F48093CC3454
:105D00002DC0E091D834F091D9348193E093D83408
:105D1000F093D9348091E1349091E23401968093EC
:105D2000E1349093E2342F5FE091E134F091E2347A
:105D30008081823209F7E091D834F091D93481938F
:105D4000E093D834F093D9348091E1349091E234E7
:105D500001968093E1349093E2342983DF91CF91CF
:105D6000089590E00E94A6460895BF92CF92DF92D8
:105D7000EF92FF920F931F93CF93DF93E091E13463
:105D8000F091E234808190E00E94A646892B29F0B0
:105D9000BB24EE24FF24870133C08BE023C09E0187
:105DA00020533040D801C70144E0880F991FAA1F33
:105DB000BB1F4A95D1F72A30310530F4790100270D
:105DC000F7FC0095102F06C0E7977E010027F7FC2F
:105DD0000095102FE80EF91E0A1F1B1F89E0B81648
:105DE00039F48CE08093CC34EE24FF24870119C071
:105DF000B3940894C11CD11CC092E134D092E23417
:105E0000C090E134D090E234F601808190E00E94AD
:105E1000B946C82FD0E0CE010E94A646892B09F0D2
:105E2000BECFB701C801DF91CF911F910F91FF90B5
:105E3000EF90DF90CF90BF9008950F931F93DF9363
:105E4000CF9300D00F92CDB7DEB70091E13410911F
:105E5000E234F8018081823229F40E945B2E22E034
:105E600030E04FC0843259F40F5F1F4F0093E1348C
:105E70001093E234015010400E94B52E0EC090E005
:105E80000E949F46892B39F0CE0101960E9485160B
:105E9000882339F434C00E94112E69837A838B835E
:105EA0009C838091CC34882351F5E091D834F091D3
:105EB000D93484EA8193E093D834F093D93469815A
:105EC0007A818B819C810E9475288091E134801BAE
:105ED00003C0F80181918F01E091D834F091D93459
:105EE0008193E093D834F093D9348091E134909148
:105EF000E2340817190768F321E030E002C020E01F
:105F000030E0C9012496CDBFDEBFCF91DF911F9154
:105F10000F910895CF93DF93EC01E881F98180819F
:105F2000843981F47396E883F98373978785908920
:105F3000009701F1DC012D913D91220F331F220FBB
:105F4000331F10C0843841F4DF011F967396E88335
:105F5000F98324E030E006C088E08093CC340E94CE
:105F6000593108C080E090E002C01D92019682176E
:105F70009307D8F3DF91CF910895EF92FF920F939B
:105F80001F93CF93DF93E82E8B01FB01019000203C
:105F9000E9F73197FE2EF61AC0912134D0912234C0
:105FA0001CC08E1581F4BE016F5F7F4FC8010E9437
:105FB0009F28F81641F48091213490912234BE013B
:105FC000681B790B0FC08881843831F0843921F047
:105FD00088E08093CC3404C063968881882309F7D5
:105FE0006FEF7FEFCB01DF91CF911F910F91FF906A
:105FF000EF9008951F93CF93DF93E9ECF2E31192B2
:1060000082E3E83DF807D9F7C091E134D091E2345A
:106010001881812F90E00E949F46892B41F01093B8
:10602000C9322196C093E134D093E23403C087E0B3
:106030008093CC34CAECD2E3E091E134F091E234C5
:1060400080810E942A2A892B71F0E091E134F0913D
:10605000E23481918993E093E134F093E23482E376
:10606000C73DD80749F7E091E134F091E2348081EF
:10607000883219F484E990E002C080E090E08093D7
:10608000D832882321F484E88093D83205C0319631
:10609000E093E134F093E2348091CC34882309F02A
:1060A00051C08091D83269EC72E30E94BD2F9C01EF
:1060B0008091CC34882309F045C08FEF2F3F3807FB
:1060C000C1F49091D832943931F48091FA33882315
:1060D00011F488E135C0892F69EC72E30E94BF2D6D
:1060E0009C018FEF2F3F380769F18091CC348823D2
:1060F00049F58091D832E091D834F091D934819328
:10610000E093D834F093D934C9010E9423288091B8
:10611000D832843949F5E091D834F091D93480E10E
:106120008193E093D834F093D93481E00E94172C06
:10613000E091E134F091E2348081893231F08EE0F7
:106140008093CC3420E030E01AC03196E093E13403
:10615000F093E234E091D834F091D93481E1819325
:10616000E093D834F093D9348091D832843829F030
:10617000843919F022E030E002C021E030E0C901AA
:10618000DF91CF911F910895E091D834F091D934E7
:106190008EE08193E093D834F093D9340895E09160
:1061A000D834F091D9348AE18193E093D834F093D4
:1061B000D9340895E091D834F091D9348CE08193AA
:1061C000E093D834F093D93408958F929F92AF9290
:1061D000BF92CF92DF92EF92FF920F931F93DF93C4
:1061E000CF93CDB7DEB76497CDBFDEBF7B018C0107
:1061F0001C8A97FF11C08DE20E94FA0FAA24BB24CB
:106200006501AE18BF08C00AD10A82E1F82E4E011E
:106210000894811C911C26C06115710581059105AA
:1062200019F05B016C01F1CF80E30E94FA0F28C0E6
:10623000080D191DC601B5012AE030E040E050E02C
:106240000E946046605DF8016083FA94C601B50162
:106250002AE030E040E050E00E946046C901DA01E7
:106260005C016D010F2D10E0A114B104C104D10433
:10627000F9F60F5F1F4FC401800F911F0E94EE0FB0
:106280006496CDBFDEBFCF91DF911F910F91FF903C
:10629000EF90DF90CF90BF90AF909F908F90089538
:1062A00098E2899FC001112484539E4F0E94DB0F06
:1062B0000895CF93DF938091B0348823D1F08EE599
:1062C0009CE10E94DB0F6091CC3470E080E090E0B4
:1062D0000E94E53084E59CE10E94DB0F6091E3348D
:1062E0007091E43480E090E00E94E53081E59CE12B
:1062F00032C00E94900F0E94900FC6EED4E302C0FD
:106300000E94FA0F89918D30D9F70E94900F26EEE6
:1063100034E304C08AE20E94FA0F9E01E90121964B
:106320008091E1349091E23402972817390790F375
:106330008DE49CE10E94DB0F0E94900F85E49CE1BC
:106340000E94DB0F6091CC3470E080E090E00E940E
:10635000E53082E49CE10E94DB0F8091CC340E9406
:10636000503181E08093C934DF91CF9108958091BD
:106370001B348F5F80931B34E091D834F091D93473
:1063800089E18193E093D834F093D93480E00E947E
:10639000172C08950F931F93E091D834F091D934BE
:1063A0008193E093D834F093D9340E943B280BE7D3
:1063B0001CE731C080E00E94172C8091CC348823E8
:1063C00099F50E943B28E091E134F091E234E081BC
:1063D000EC3231F4E091D834F091D934108307C015
:1063E000EB3311F5E091D834F091D93400838091EA
:1063F000E1349091E23401968093E1349093E23459
:106400008091D8349091D93401968093D834909368
:10641000D9340E943B28E091E134F091E234E081EC
:10642000ED3011F0EA3331F61F910F91089583E4B6
:106430000E94CA31089583E00E94CA310895E09114
:10644000D834F091D93483E28193E093D834F09337
:10645000D9340E943B280E94FA2F08951F931CE70D
:106460000E943B280E94FA2F8091CC348823E1F4CB
:106470000E943B28E091E134F091E23480818C323B
:1064800099F4E091D834F091D9341193E093D83451
:10649000F093D9348091E1349091E2340196809365
:1064A000E1349093E234DCCF1F91089581E0809332
:1064B000FA33E091D834F091D93489E08193E093B4
:1064C000D834F093D9340E942E321092FA330895C2
:1064D000E091D834F091D9348DE08193E093D834B1
:1064E000F093D9340E942E320895E091D834F0917F
:1064F000D93485E08193E093D834F093D9340E9465
:106500003B280E94FA2F019719F082E08093CC3447
:106510000895E091D834F091D93486E18193E093E5
:10652000D834F093D9340E943B28E091E134F091C3
:10653000E2348081823221F50E945B2E8091CC343E
:10654000882301F5E091E134F091E23480818C32CE
:1065500021F082E08093CC340895E091D834F0911A
:10656000D9348CE78193E093D834F093D934809177
:10657000E1349091E23401968093E1349093E234D7
:106580000E942E3208951F9381E080932736E09178
:10659000D834F091D93484E08193E093D834F093E7
:1065A000D9340E943B280E94FA2F182F0E943B28C2
:1065B000113059F4E091E134F091E2348191E093AB
:1065C000E134F093E2348D3311F083E02EC0E0919A
:1065D000D834F091D93489E78193E093D834F0939B
:1065E000D93481E00E94172C8091CC348823C9F5DE
:1065F0000E943B288DEC90E20E94D128892BA1F0CB
:10660000E091D834F091D93487E38193E093D83482
:10661000F093D9340E943B2881E00E94172C80918E
:10662000CC348823F1F404C081E18093CC3419C0C8
:106630000E943B2880ED90E20E94D128892B79F0BE
:10664000E091D834F091D9348AE38193E093D8343F
:10665000F093D9340E943B2881E00E94172C1092BD
:1066600027361F910895E091D834F091D93485E10F
:106670008193E093D834F093D9340E943B288091E1
:106680001B348F5F80931B3481E00E94172C809114
:10669000CC34882309F07CC00E943B2885ED90E231
:1066A0000E94D128892BB9F1E091D834F091D934E6
:1066B00088E38193E093D834F093D9340E943B2847
:1066C000E091E134F091E234808190E0C0970A9744
:1066D000D8F4E091D834F091D93488EA8193E093EA
:1066E000D834F093D9340E94EB279C01009719F419
:1066F00082E18093CC348091CC34882309F048C067
:10670000C9010E9423280BC00E94F9288091CC3433
:10671000882329F0089580E18093CC3408950E9465
:106720003B288AED90E20E94D128892B89F1E091E3
:10673000D834F091D93489E38193E093D834F0933D
:10674000D9340E943B28E091E134F091E234808119
:1067500090E0C0970A97D0F4E091D834F091D93402
:1067600088EA8193E093D834F093D9340E94EB27E0
:106770009C01009719F482E18093CC348091CC3451
:10678000882331F4C9010E94232808950E94F92822
:106790000895FF920F931F93E091D834F091D9346C
:1067A00083E18193E093D834F093D9340E943B285D
:1067B00081E00E94172C8091CC34882309F056C0C8
:1067C0000E943B288FED90E20E94D128892B19F07E
:1067D0000E94A92D0CC084EE90E20E94D128892B42
:1067E00019F00E94AD2D03C08FE08093CC348091CE
:1067F000CC348823D9F50E943B289CE7F92E08EA7F
:1068000012E12DC0E091D834F091D934F192E093A7
:10681000D834F093D9348091E1349091E2340196E8
:106820008093E1349093E2340E943B28E091D83485
:10683000F091D9340193E093D834F093D9340E9485
:10684000EB279C01009711F41093CC348091CC3449
:10685000882361F4C9010E942E280E943B28E09100
:10686000E134F091E23480818C3261F21F910F911A
:10687000FF900895DF92EF92FF920F931F93CF93B3
:10688000DF938B017A01C091D834D091D934DE01E5
:106890008D93A093D834B093D934E091E134F09142
:1068A000E2348081883239F580E189831196A093A2
:1068B000D834B093D9348091E1349091E234019688
:1068C0008093E1349093E2348CE7D82EF7018191E4
:1068D0007F010E94172C8091CC348823D9F5015078
:1068E0001040E091E134F091E23401151105C1F05E
:1068F00080818C3211F082E017C0E091D834F091A1
:10690000D934D192E093D834F093D9348091E134E2
:106910009091E23401968093E1349093E234D6CFA3
:106920008081893221F08EE08093CC3413C0E091D5
:10693000D834F091D93481E18193E093D834F09345
:10694000D9348091E1349091E23401968093E1341E
:106950009093E234DF91CF911F910F91FF90EF90D0
:10696000DF900895DF93CF930F92CDB7DEB791E01C
:10697000998361E070E0AE014F5F5F4F0E943A344F
:1069800081E00F90CF91DF91089583E10E94B234AE
:10699000089582E10E94B23408958AE00E94B234E0
:1069A000089580E10E94B23408958FE00E94B234CD
:1069B000089589E00E94B23408958EE00E94B234B6
:1069C00008958DE00E94B23408958BE00E94B234A5
:1069D00008958CE00E94B234089583E00E94B2349E
:1069E00090E0089581E10E94B23408958BE00E9406
:1069F000B234089587E00E94B23490E0089586E0B2
:106A00000E94B23490E0089585E00E94B23490E094
:106A1000089584E00E94B23490E0089582E00E94DC
:106A2000B23490E008950E94B2340E943B28E09175
:106A3000E134F091E2348191E093E134F093E23477
:106A40008D3321F083E08093CC340895E091D834E5
:106A5000F091D93489E78193E093D834F093D93415
:106A600081E00E94172C08958DE10E94133508954E
:106A70008CE10E94133508958BE10E94133508952F
:106A8000CF93DF93C091D834D091D93486E38883F3
:106A90008091D8349091D93401968093D8349093D2
:106AA000D9348AEE90E20E94D128892B19F00E94F5
:106AB0000E3595C08FEE90E20E94D128892B19F0F7
:106AC0000E9409358CC083EF90E20E94D128892B67
:106AD00019F00E94ED3483C088EF90E20E94D12823
:106AE000892B19F00E9404357AC08CEF90E20E9445
:106AF000D128892B19F00E94FF3471C080E091E207
:106B00000E94D128892B19F00E94FA3468C084E0D1
:106B100091E20E94D128892B19F00E94DD345FC0D8
:106B200089E091E20E94D128892B19F00E94E1347A
:106B300056C08EE091E20E94D128892B19F00E9464
:106B4000E5344DC082E191E20E94D128892B19F0F1
:106B50000E94D53444C089E191E20E94D128892B5A
:106B600019F00E94D1343BC080E291E20E94D1280A
:106B7000892B19F00E94D93432C085E291E20E943B
:106B8000D128892B19F00E94F23429C08AE291E2BF
:106B90000E94D128892B19F00E94C93420C080E3BB
:106BA00091E20E94D128892B19F00E94C53417C0A8
:106BB00086E391E20E94D128892B19F00E94CD34FE
:106BC0000EC08AE391E20E94D128892B19F00E941D
:106BD000E93405C0C093D834D093D93480E0DF9134
:106BE000CF9108951F93CF93DF93DB01EC018A814E
:106BF0006AE00E944046805DFD0181938A810E9487
:106C00004046905D11969C93DF0111961AE3118323
:106C1000AD014F5F5F4F89810E944046805D1196B4
:106C20008C93FA01319689810E944046905DDA0189
:106C300011969C93DF0111961183FD013196888195
:106C40000E944046805D11968C9388810E94404648
:106C5000905D91831282DF91CF911F9108950895E5
:106C60000895E091D834F091D93480818E3719F0AD
:106C70008F3761F406C03196E093D834F093D9345D
:106C800008953296E093D834F093D934089586E885
:106C900095E38093D8349093D9340E9431361DC047
:106CA0000E943136E091D834F091D9348191E0934B
:106CB000D834F093D93490E001979C01220F331F10
:106CC000280F391F220F331F220F331F2C5B334F26
:106CD000F90185919491FC011995E091D834F091D6
:106CE000D93480818D3721F08091CC348823C1F252
:106CF00008958AE0809382358091D734882371F09B
:106D00001092D73489E38093CC348091D83390911A
:106D1000D933809384359093853581E008950F931E
:106D20001F93DF93CF930F920F92CDB7DEB70E94E0
:106D30009D3C809121349091223489839A838E01E5
:106D40000F5F1F4F03C0C8010E948A2FE981FA819B
:106D500080818823C1F70F900F90CF91DF911F9111
:106D60000F9108950E948F361092D7341092833578
:106D70008AE0809382351092C9341092C034109208
:106D8000C1340895DF93CF93CDB7DEB76497CDBFFD
:106D9000DEBF2091DC343091DD348091D43390918A
:106DA000D5332817390791F080E99CE10E94DB0F69
:106DB000CE0101960E941A108981893711F0893518
:106DC00049F40E94B23C8EE79CE102C086E69CE159
:106DD0000E94DB0F6496CDBFDEBFCF91DF91089597
:106DE00007C03196E093D932F093DA320E94FA0F5D
:106DF000E091D932F091DA3280818D3791F70895A0
:106E00000F931F93CF93DF93A091D932B091DA32D1
:106E1000FD012191E093D932F093DA322633F1F17A
:106E2000273330F42A3021F12C3009F04DC026C030
:106E30002E37D1F02F3721F0243409F045C01BC084
:106E400011968C913196E093D932F093DA32C0E00A
:106E5000D0E0082F10E004C080E20E94FA0F2196D3
:106E6000C017D107CCF340C080E20E94FA0F3CC0AB
:106E70008DEE9CE105C08BEE9CE102C086EE9CE1AC
:106E80000E94DB0F8091D9329091DA320196809383
:106E9000D9329093DA320E94F03626C011962C91A6
:106EA0003196E093D932F093DA3230E0215030401D
:106EB000C901880F991F820F931F880F991F880F90
:106EC000991F8A5A944F0EC030E021503040C901BA
:106ED000880F991F820F931F880F991F880F991F82
:106EE0008A5B934F0E94DB0FDF91CF911F910F912F
:106EF00008951F9390E00196E091D932F091DA3233
:106F0000E80FF91FE093D932F093DA321191E09350
:106F1000D932F093DA320CC0E091D932F091DA3202
:106F20008191E093D932F093DA320E94FA0F115036
:106F3000112391F71F91089580E00E9479370895F9
:106F400084E00E947937089584E00E94793708959B
:106F50000F931F93CF93DF93E091D932F091DA3200
:106F6000818192813396E093D932F093DA32C091E5
:106F70002134D0912234C80FD91F8E01025F1F4FD8
:106F80008981882311F00E94FA0F2196C017D1073A
:106F9000B9F7DF91CF911F910F9108950E94A83703
:106FA0000895E091D834F091D93482819F01280F5F
:106FB000311D2093D8333093D933819191918093AF
:106FC000E3349093E434E093D834F093D93480914F
:106FD000CD33882389F08BE50E94FA0F6091E3346A
:106FE0007091E43480E090E00E94E5308DE50E94ED
:106FF000FA0F80E20E94FA0F0895E091D932F091E1
:10700000DA32618172813396E093D932F093DA32C9
:10701000882777FD8095982F0E94E53008955CC001
:107020000E94D1378091D8349091D93401968093C1
:10703000D8349093D9343AC00E943136E091D83494
:10704000F091D9348191E093D834F093D9348F30D2
:1070500041F40E94E31F8091CC34882309F041C0A1
:1070600082E190E001979C01220F331F280F391F06
:10707000220F331F220F331F2C5B334FF9018591F1
:107080009491FC0119958091CC34882351F580911D
:107090008235882319F08150809382358091823522
:1070A000882321F40E9479368823D9F4E091D834DA
:1070B000F091D93480818D3709F0BECF9F012F5FC9
:1070C0003F4F8091D4339091D5332817390749F039
:1070D0002093D8343093D9348091CC34882309F468
:1070E0009FCF08958091C934882359F480918435C5
:1070F000909185358093D8349093D9340E940F387D
:10710000089585E28093CC340E94593108950E94FD
:10711000900F0E94B23681E08093B0342091DC342D
:107120003091DD348091D4339091D53328173907CD
:1071300029F487EC9CE10E94DB0F08952093D8345A
:107140003093D9342093D8333093D9330E940F38F9
:107150008091CC34882311F00E9459310E94900F05
:1071600008950F931F93DF93CF93CDB7DEB72F977B
:10717000CDBFDEBFE091D932F091DA3281819281C8
:107180003396E093D932F093DA328E010F5F1F4FBE
:10719000B8010E947316C8010E94EE0F2F96CDBF52
:1071A000DEBFCF91DF911F910F910895E091D93209
:1071B000F091DA32E081E93870F4E13821F0E23818
:1071C000D9F1E43819F40E94A8370895E33869F535
:1071D0000E94B1380895E93A60F5E13A19F40E9445
:1071E000A4370895E23A19F40E949C370895E83ACA
:1071F00019F40E94FD370895E43A19F40E94A0376B
:107200000895E43991F40E94A83707C0E7FF03C04E
:107210000E94D63802C00E940037E091D932F09126
:10722000DA32E081ED3791F7089588E08093CC342D
:10723000089588E08093CC3408956F927F928F9266
:107240009F92AF92BF92CF92DF92EF92FF920F93F5
:107250001F93DF93CF93CDB7DEB7CF58D040CDBFCC
:10726000DEBF0E94DD27E091E134F091E23410812D
:10727000812F90E00E949F46892B09F43EC180E453
:1072800091E20E94D128892B09F43EC00E94900F00
:1072900086E491E20E94EE0FEE24FF248E010F5F40
:1072A0001F4FC70165E070E00E944C46892B11F426
:1072B0000E94900FC701B8010E947316898188232C
:1072C00001F1F80101900020E9F73197E01BF10B83
:1072D0003E9738F01F860EC0C80167E571E20E9434
:1072E000D146F80101900020E9F73197E01BF10B3E
:1072F0003E9790F3C8010E94EE0F0894E11CF11C28
:10730000D0CF0E94900FF6C089E591E20E94D1286B
:10731000892B09F471C00E94900F109121340091C3
:1073200022348EE591E20E94EE0F812F902F6C01A6
:1073300076010894E11CF11CAA24BB2490E1892E5B
:10734000912C54C0C50183709070892B11F40E9458
:10735000900FF60180818438D1F4C7010E94EE0FAE
:10736000F70101900020E9F73197EE19FF09840138
:107370000E1B1F0B06C087E591E20E94EE0F015025
:10738000104001151105B9F783E791E224C0843953
:1073900009F0B0C0C7010E94EE0F88E791E20E9499
:1073A000EE0F8AE791E20E94EE0FF70101900020B4
:1073B000E9F73197EE19FF0984010E1B1F0B06C078
:1073C00087E591E20E94EE0F015010400115110572
:1073D000B9F78CE791E20E94EE0F0894A11CB11C52
:1073E00083E190E0C80ED91EE80EF91EF6018081F7
:1073F000882309F0A7CF7EC08FE791E20E94D128B1
:10740000892B09F473C0A090D932B090DA32EE24FF
:10741000FF24870180E1882E912C8C0E9D1EB2E105
:107420006B2E712C6C0E7D1E85E19DE10E94DB0FA1
:10743000C801B7010E94E53082E19DE10E94DB0FA7
:107440008E2D0E945B11AB01BC01411551056105F8
:107450007105A9F1C40120E830E00E947414F40120
:10746000C080D1806092D9327092DA32FFEFCF16AD
:10747000FFEFDF0619F485E09DE123C080E20E9462
:10748000FA0FB60180E090E00E94E5308091D93299
:107490009091DA3201968093D9329093DA3207C014
:1074A000E7FF03C00E94D63802C00E940037E09177
:1074B000D932F091DA32E081ED3791F704C081EFF3
:1074C0009CE10E94DB0F0E94900F0894E11CF11CCC
:1074D000011D111D83E0E816F1040105110509F0F5
:1074E000A3CFA092D932B092DA3204C085E891E2FB
:1074F0000E94EE0F0E94900FACC0812F90E0C097C9
:10750000E091DC34F091DD342091D4333091D533E7
:107510000A97A0F5E217F30709F49BC00E94EB2736
:107520008093C6349093C7340E94DD27E091E13404
:10753000F091E23480818D32C1F43196E093E134F0
:10754000F093E2340E94DD27E091E134F091E234DF
:10755000808190E0C0970A9718F40E94EB2709C039
:1075600080917E3590917F3504C08091C634909192
:10757000C7348093B1349093B23412C0E217F3074A
:1075800009F467C080917E3590917F358093B13446
:107590009093B234808191818093C6349093C734A4
:1075A0002091C6343091C7348091B1349091B23477
:1075B0008217930708F44DC0C9010E94CE3C809306
:1075C000D9329093DA320E94900FE091D932F09143
:1075D000DA328091D4339091D533E817F907C8F5A2
:1075E00001911191E093D932F093DA328091B13464
:1075F0009091B2348017910760F180E20E94FA0FF7
:10760000B80180E090E00E94E5308091D9329091FD
:10761000DA3201968093D9329093DA3207C0E7FFCD
:1076200003C00E94D63802C00E940037E091D932D0
:10763000F091DA32E081ED3791F70E94900F80915E
:10764000D9329091DA3201968093D9329093DA321E
:10765000BCCFC157DF4FCDBFDEBFCF91DF911F91B0
:107660000F91FF90EF90DF90CF90BF90AF909F90E1
:107670008F907F906F900895DF92EF92FF920F931B
:107680001F937C018B01DC0113968C9113976AE0A8
:107690000E944046805DF801819313968C910E9470
:1076A0004046905DD80111969C9320E2D22ED18263
:1076B000CF0102966BEC71E20E94DC46F801D682A3
:1076C000D70115968C91159764E60E944046892F44
:1076D0006AE00E944046805D878315968C9164E63F
:1076E0000E944046892F6AE00E944046905D908744
:1076F00011861F910F91FF90EF90DF9008958FEC0E
:1077000091E20E94D128892B19F00E941D394AC0AC
:1077100084ED91E20E94D128892B19F00E948738CC
:1077200041C088ED91E20E94D128892B19F00E9476
:10773000C23638C08CED91E20E94D128892B19F015
:107740000E9472382FC081EE91E20E94D128892BCD
:1077500019F00E948F3626C087EE91E20E94D12850
:10776000892B19F00E94D93B1DC08CEE91E20E943A
:10777000D128892B19F00E94331A14C081EF91E2AD
:107780000E94D128892B19F00E94491C0BC086EF5A
:1077900091E20E94D128892B19F420E030E004C046
:1077A0000E942A3C21E030E0C9010895089508951F
:1077B00008950E94900F8DE69DE10E94DB0F60917D
:1077C000CA347091CB342091D4333091D533621BBD
:1077D000730B882777FD8095982F0E94E53081E60E
:1077E0009DE10E94DB0F0E94900F8FE49DE10E94BB
:1077F000DB0F6091D1347091D23420917C3530917F
:107800007D35621B730B882777FD8095982F0E942A
:10781000E53083E49DE10E94DB0F0E94900F84E23B
:107820009DE10E94DB0F6091783570917935209150
:10783000193430911A34621B730B882777FD8095B9
:10784000982F0E94E53088E19DE10E94DB0F0E94A5
:10785000900F08951F930E94DD27E091E134F0918D
:10786000E23480818D3081F50E94EF15182F8D351F
:1078700028F48A3558F48535C9F405C08F3FB1F432
:1078800081E09EE152C08AEE9DE14FC084ED9DE112
:107890000E94DB0F1A3511F480E305C01B3511F48B
:1078A00081E301C082E30E94FA0F0AC08BEB9DE1E5
:1078B0000E94DB0F612F70E080E090E00E94E530D5
:1078C0008EE20E94FA0F33C08DEF91E20E94D12820
:1078D000892B19F08FEF90E023C081E092E20E94A3
:1078E000D128892B19F085E590E01AC084E092E256
:1078F0000E94D128892B19F08AE590E011C088E018
:1079000092E20E94D128892B19F08BE590E008C003
:107910008CE092E20E94D128892B29F08CE590E03E
:107920000E949D1A04C08EE79DE10E94DB0F1F910B
:10793000089508950895089508958AE695E36DEDF4
:1079400072E34CE30E94642786E695E36BEF73E3F2
:107950004EE10E946A271092CE331092B3341092F7
:10796000E03408950E94340F10927E3510927F35D6
:10797000109220340895FB01E80FF91FDB0102C0CB
:1079800081918D938091D4339091D533E817F90785
:10799000B8F3A093D433B093D53308959C01E0910C
:1079A000DC34F091DD34808191818217930714F0EB
:1079B000CF0108958281E80FF11DF5CFE091DC340D
:1079C000F091DD344091D4335091D53320E030E054
:1079D0000BC0208131812115310519F420E030E000
:1079E00006C08281E80FF11DE417F50791F7C90180
:1079F00008959C0180917E3590917F358217930781
:107A0000A0F1E091DC34F091DD34DF014D915D9126
:107A10004217530724F04217530739F507C08281F4
:107A2000E82FF0E03297EA0FFB1FEFCF8C91DF01D8
:107A3000A80FB11D02C08D9181938091D433909194
:107A4000D533A817B907B8F3E093D433F093D533FF
:107A500080917E3590917F354817590731F40E9407
:107A6000DE3C80937E3590937F350895A091D4338A
:107A7000B091D533FD01E80FF91F8091CA34909180
:107A8000CB348E179F0720F489E08093CC3408957F
:107A9000E093D433F093D5336150704004C08C919F
:107AA000808331971197A617B707C9F70895DC01AE
:107AB00080918835282F30E086E895E38093D8348C
:107AC0009093D9340CC0E091D834F091D93481919D
:107AD0008D93E093D834F093D93421503040211560
:107AE000310589F70895CF93DF93EC0180918835B4
:107AF00090E0BE010E94363D8091CC34882319F479
:107B0000CE010E94573DDF91CF9108954091D4332B
:107B10005091D533809188359A01280F311D80917D
:107B2000CA349091CB348217930780F0CA010E9427
:107B3000573D209188358091D4339091D533820F71
:107B4000911D8093D4339093D533089589E0809329
:107B5000CC340895CF93DF93EC018A81282F30E055
:107B600080918835281B31092115310501F137FF36
:107B70000CC088279927821B930BBE010E94363DBB
:107B80008091CC348823B1F412C0DE01A20FB31F60
:107B9000FE0102C08D9181938091D4339091D533B1
:107BA000A817B907B8F3E093D433F093D533CE01D7
:107BB0000E94573DDF91CF910895CF93DF9381E0ED
:107BC0008093C93486E895E38093D8349093D93470
:107BD000C0918635D091873580917E3590917F35E3
:107BE0008C179D0738F40E94863DC0937E35D09354
:107BF0007F3518C0E091DC34F091DD3480819181D3
:107C00008C179D0724F0C817D90749F404C0828156
:107C1000E80FF11DF3CFCF010E94AA3D03C0CF01B1
:107C20000E94733DDF91CF91089590E00197FC0190
:107C3000EE0FFF1FE80FF91FEE0FFF1FEE0FFF1FE4
:107C4000EC5BF34F85919491009711F0FC0119952D
:107C50000895EF92FF920F931F93CF93DF9320919C
:107C60006B3581E090E0821B9109880F991F880F86
:107C7000991FC0916C35D0916D35C81BD90B2881E7
:107C800039814A815B81CA01AA27BB27F9010BB65A
:107C90008BBF819190810BBE7C0100E010E02E5FD4
:107CA0003F4F4F4F5F4FCA01AA27BB27F9010BB6C1
:107CB0008BBF219130810BBEC901A0E0B0E0DC0197
:107CC000992788278E0D9F1DA01FB11F8883998338
:107CD000AA83BB83DF91CF911F910F91FF90EF900B
:107CE0000895CF93DF9320916B3581E090E0821B64
:107CF0009109880F991F880F991FC0916C35D091F9
:107D00006D35C81BD90B88819981AA81BB819D01E2
:107D100044275527FC010BB62BBF80810BBE90E09A
:107D2000A0E0B0E088839983AA83BB83DF91CF91E1
:107D30000895CF93DF9320916B3581E090E0821B13
:107D40009109880F991F880F991FC0916C35D091A8
:107D50006D35C81BD90B88819981AA81BB819D0192
:107D600044275527FC010BB62BBF819190810BBE98
:107D7000A0E0B0E088839983AA83BB83DF91CF9191
:107D8000089520916B3581E090E0821B9109880F66
:107D9000991F880F991FE0916C35F0916D35E81BA4
:107DA000F90B80819181A281B38180959095A095F6
:107DB000B09580839183A283B383089520916B351E
:107DC00081E090E0821B9109880F991F880F991F0D
:107DD000E0916C35F0916D35E81BF90B8081918154
:107DE000909581959F4FAA2797FDA095BA2F8083E4
:107DF0009183A283B383089589E28093CC3408955C
:107E00006F927F928F929F92AF92BF92CF92DF92AA
:107E1000EF92FF920F931F93CF93DF938AE695E340
:107E200068E30E949D27AC01CB01DA015C016D0182
:107E300020916B3581E090E0821B9109880F991F9A
:107E4000880F991FC0916C35D0916D35C81BD90B27
:107E5000288139814A815B81D7FE04C0EE24FF244A
:107E6000870126C039014A0171E0E72EF12C012D6E
:107E7000112D19C0C50181709070892B41F0C80186
:107E8000B7019301A4010E9421467B018C01B3013B
:107E9000C4019301A4010E9421463B014C01D594E9
:107EA000C794B794A794A114B104C104D10411F7E5
:107EB000E882F9820A831B83DF91CF911F910F9192
:107EC000FF90EF90DF90CF90BF90AF909F908F90FA
:107ED0007F906F9008958AE695E368E30E949D275E
:107EE00040916B3521E030E0241B3109220F331F14
:107EF000220F331FE0916C35F0916D35E21BF30BCF
:107F0000208131814281538126173707480759075D
:107F100049F081E090E0A0E0B0E080839183A2830B
:107F2000B3830895108211821282138208958AE623
:107F300095E368E30E949D2740916B3521E030E096
:107F4000241B3109220F331F220F331FE0916C35A0
:107F5000F0916D35E21BF30B208131814281538119
:107F6000261737074807590749F481E090E0A0E059
:107F7000B0E080839183A283B3830895108211823D
:107F80001282138208958AE695E368E30E949D2792
:107F900040916B3521E030E0241B3109220F331F63
:107FA000220F331FE0916C35F0916D35E21BF30B1E
:107FB00020813181428153812617370748075907AD
:107FC0004CF081E090E0A0E0B0E080839183A28358
:107FD000B3830895108211821282138208958AE673
:107FE00095E368E30E949D2740916B3521E030E0E6
:107FF000241B3109220F331F220F331FE0916C35F0
:10800000F0916D35E21BF30B208131814281538168
:1080100062177307840795074CF081E090E0A0E0B9
:10802000B0E080839183A283B3830895108211828C
:108030001282138208958AE695E368E30E949D27E1
:1080400040916B3521E030E0241B3109220F331FB2
:10805000220F331FE0916C35F0916D35E21BF30B6D
:10806000208131814281538162177307840795070C
:108070004CF481E090E0A0E0B0E080839183A283A3
:10808000B3830895108211821282138208958AE6C2
:1080900095E368E30E949D2740916B3521E030E035
:1080A000241B3109220F331F220F331FE0916C353F
:1080B000F0916D35E21BF30B2081318142815381B8
:1080C00026173707480759074CF481E090E0A0E0F5
:1080D000B0E080839183A283B383089510821182DC
:1080E0001282138208950F931F938AE695E368E343
:1080F0000E949D279B01AC0160916B3581E090E06F
:10810000861B9109880F991F880F991F00916C3564
:1081100010916D35081B190BF80160817181828106
:1081200093810E942146F801608371838283938347
:108130001F910F9108950F931F938AE695E368E3CB
:108140000E949D279B01AC0160916B3581E090E01E
:10815000861B9109880F991F880F991F00916C3514
:1081600010916D35081B190BF801608171818281B6
:1081700093810E948246F801608371838283938396
:108180001F910F9108958AE695E368E30E949D2769
:1081900040916B3521E030E0241B3109220F331F61
:1081A000220F331FE0916C35F0916D35E21BF30B1C
:1081B0002081318142815381261B370B480B590B9B
:1081C000208331834283538308958AE695E368E3ED
:1081D0000E949D2740916B3521E030E0241B31093E
:1081E000220F331F220F331FE0916C35F0916D3554
:1081F000E21BF30B2081318142815381260F371F0F
:10820000481F591F208331834283538308958AE690
:1082100095E368E30E949D2740916B3521E030E0B3
:10822000241B3109220F331F220F331FE0916C35BD
:10823000F0916D35E21BF30B208131814281538136
:1082400026233723482359232083318342835383B2
:1082500008958AE695E368E30E949D2740916B3577
:1082600021E030E0241B3109220F331F220F331F7E
:10827000E0916C35F0916D35E21BF30B208131817B
:1082800042815381262B372B482B592B2083318356
:108290004283538308958AE695E368E30E949D270D
:1082A00040916B3521E030E0241B3109220F331F50
:1082B000220F331FE0916C35F0916D35E21BF30B0B
:1082C000208131814281538126273727482759272A
:1082D000208331834283538308958AE695E368E3DC
:1082E0000E949D27CB010895CF92DF92EF92FF92DB
:1082F0000F931F938AE695E368E30E949D276B0125
:108300007C01C114D104E104F104F9F020916B3532
:1083100081E090E0821B9109880F991F880F991FB7
:1083200000916C3510916D35081B190BF8016081B7
:10833000718182819381A70196010E948246F80192
:10834000208331834283538305C08AE18093CC34F8
:108350000E9459311F910F91FF90EF90DF90CF90C5
:1083600008950F931F93682F86E695E347E10E94D7
:1083700083273DC08091CC348823F1F5E0916835A6
:10838000F0916935E90FF11D429152914031A1F10F
:10839000242F30E0207F3070852F90E0807F907018
:1083A000821793074CF1413169F4503159F486E654
:1083B00095E368E30E94702786E695E368E30E94F0
:1083C00070271AC086E695E368E30E947027082F9D
:1083D00086E695E368E30E947027182F86E695E30A
:1083E000602F47E10E948327812F0E94153E9091C4
:1083F0006735923008F0BECF1F910F9108958933F1
:1084000028F4873360F4813141F409C08A3339F0AC
:108410008A3318F08A57863010F080E0089581E1A1
:108420000E94B14181E00895CF93DF93843861F0D9
:10843000853820F4833809F081C070C0843979F11F
:10844000843A09F07BC014C0E091D834F091D9345B
:10845000818192813396E093D834F093D9340F968A
:108460000E945F0FFC0140815181628173816CC069
:10847000E091D834F091D934418152816381748183
:108480003596E093D834F093D93435978581369674
:10849000E80FF11DE093D834F093D93455C0E09142
:1084A000D834F091D934818192813396E093D834D5
:1084B000F093D9340F960E945F0FFC01C081D181E7
:1084C0008091D8349091D93401968093D834909388
:1084D000D9340E94AC428091D8349091D93401961D
:1084E0008093D8349093D9348AE695E368E30E9468
:1084F0009D27FB0188819981E817F90720F089E120
:108500008093CC3426C0EE0FFF1FEE0FFF1FEC0F41
:10851000FD1F428153816481758116C0E091D8347A
:10852000F091D934818192813396E093D834F093DD
:10853000D9340E94A310AB01BC0106C088E080932F
:10854000CC340E94593105C08AE695E327E10E94A8
:10855000BD27DF91CF9108951F9380E10E94B14123
:108560000E943136E091D834F091D9348081803145
:1085700041F43196E093D834F093D9340E94AC4260
:1085800018C087FF07C00E9414428091CC34882312
:1085900039F319C00E945045182F8091CC3488239C
:1085A00091F4812F0E94FF41882369F4812F0E945A
:1085B000B1418091D8349091D93401968093D834C8
:1085C0009093D934CDCF1F910895EF92FF920F93DE
:1085D0001F93CF93DF930E94AC4220916B3581E0D3
:1085E00090E0821B9109880F991F880F991FC091F5
:1085F0006C35D0916D35C81BD90BE880F9800A81A4
:108600001B81E114F1040105110569F48EE491E682
:10861000ACEBB0E08093102290931122A093122231
:10862000B093132228C06091102270911122809182
:108630001222909113222DE036E649E150E00E948B
:108640002146615A7C408149934C6093102270937B
:1086500011228093122290931322A80197010E9465
:1086600060469B01AC012F5F3F4F4F4F5F4F288308
:1086700039834A835B83DF91CF911F910F91FF90E4
:10868000EF900895AF92BF92CF92DF92EF92FF9258
:108690000F931F930E94AC4220916B3581E090E0D4
:1086A000821B9109880F991F880F991FE0916C35E3
:1086B000F0916D35E81BF90BA080B180C280D380AA
:1086C000E12CF12C012DA0E41A2F07C072E01695C1
:1086D0000795F794E7947A95D1F7AE14BF04C006D6
:1086E000D106A0F320E030E040E050E024C0D80103
:1086F000C701820F931FA41FB51FA816B906CA068B
:10870000DB0670F0A81AB90ACA0ADB0AD801C70149
:10871000880F991FAA1FBB1F280F391F4A1F5B1FF5
:10872000569547953795279582E016950795F794C6
:10873000E7948A95D1F7E114F10401051105B9F622
:108740002A153B054C055D0520F42F5F3F4F4F4F29
:108750005F4F20833183428353831F910F91FF909A
:10876000EF90DF90CF90BF90AF9008951F93DF936D
:10877000CF9300D00F92CDB7DEB7182F0E94AC4236
:1087800020916B3581E090E0821B9109880F991F41
:10879000880F991FE0916C35F0916D35E81BF90B4E
:1087A0006081718182819381123039F0143071F0CF
:1087B000113099F40E94D5150BC00E94B815698339
:1087C0007A838B839C830E94900F0EC00E94B51405
:1087D00069837A838B839C8307C083E08093CC3446
:1087E00019821A821B821C8229813A814B815C8109
:1087F00060916B3581E090E0861B9109880F991F8D
:10880000880F991FE0916C35F0916D35E81BF90BDD
:1088100020833183428353832496CDBFDEBFCF9123
:10882000DF911F91089584E00E94B643089582E08D
:108830000E94B643089581E00E94B64308950E94C5
:10884000AC4220916B3581E090E0821B9109880F4A
:10885000991F880F991FE0916C35F0916D35E81BD9
:10886000F90BA081B1818D919D910D90BC91A02DAE
:1088700080839183A283B38308950E94AC422091A8
:108880006B3581E090E0821B9109880F991F880F5A
:10889000991FE0916C35F0916D35E81BF90BA081C3
:1088A000B1818D919C91A0E0B0E080839183A283FF
:1088B000B38308950E94AC4220916B3581E090E033
:1088C000821B9109880F991F880F991FE0916C35C1
:1088D000F0916D35E81BF90BA081B1818C9190E08E
:1088E000A0E0B0E080839183A283B38308950E94C7
:1088F000AC4208950E94AC4220916B3581E090E03B
:10890000821B9109880F991F880F991FE0916C3580
:10891000F0916D35E81BF90B80819181A281B381C3
:108920000097A105B10529F41082118212821382E9
:108930000895B7FF05C08FEF9FEFAFEFBFEF04C003
:1089400081E090E0A0E0B0E080839183A283B383D4
:1089500008950E94AC4220916B3581E090E0821B2B
:108960009109880F991F880F991FE0916C35F0913C
:108970006D35E81BF90B2081318137FF03C030953D
:1089800021953F4FC901AA2797FDA095BA2F808353
:108990009183A283B3830895CF93DF93843861F0EA
:1089A000853820F4833809F06DC05CC08439D1F07B
:1089B000843A09F067C014C0E091D834F091D934FA
:1089C000818192813396E093D834F093D9340F9615
:1089D0000E945F0FAC01662757FD6095762F58C047
:1089E0008AE351C0E091D834F091D93481819281E9
:1089F0003396E093D834F093D9340F960E945F0FEA
:108A0000FC01C081D1818091D8349091D9340196F4
:108A10008093D8349093D9340E94AC428091D8345A
:108A20009091D93401968093D8349093D9348AE6C2
:108A300095E368E30E949D278881998168177907EB
:108A400020F089E18093CC3428C02296660F771FEE
:108A5000660F771FC60FD71FAE01662757FD6095BB
:108A6000762F16C0E091D834F091D934818192816B
:108A70003396E093D834F093D9340E942311AB019C
:108A8000BC0106C088E08093CC340E94593105C0F7
:108A90008AE695E327E10E94BD27DF91CF910895F3
:108AA000863309F071C0E091D834F091D934319611
:108AB000E093D834F093D934319781813396E093A1
:108AC000D834F093D93433978A30F1F18B3098F45D
:108AD000853059F1863040F4833021F18430F8F448
:108AE000823009F041C039C08730B9F1873000F1D8
:108AF0008930D1F520C08F3009F1803138F48D30C4
:108B000061F18E3050F58B3079F527C0813149F114
:108B10008131B8F08231D9F0833131F51BC00E9428
:108B2000A94422C00E9442431FC00E94E5421CC0CB
:108B30000E947A4419C00E945A4416C00E943D44C3
:108B400013C00E941F4410C00E941B440DC00E940D
:108B500017440AC00E94134407C089E28093CC34B2
:108B600003C083810E94CC448091D8349091D93441
:108B700001968093D8349093D9340E943136E09195
:108B8000D834F091D934808108958FEF8093E00636
:108B90008093200780EF80930007E0E4F4E089E011
:108BA0008093400486E0818389E4808781878FEF0A
:108BB00093E08483958380E090E28683978380911D
:108BC0005D04887F80935D0410925E0410925F04C0
:108BD00080915C0480788F6380935C0480915D0455
:108BE00087FFFCCF0895FC01E050F04C60830895AE
:108BF000FC01E050F04C80810895DC01CB01F89439
:108C00008050904CAF4FBF4F9D0144275527FC012A
:108C10000BB62BBF80810BBE789408950F931F93E2
:108C20006050704C8F4F9F4FF8948C012227332750
:108C3000FB010BB60BBF40830BBE78941F910F91C5
:108C40000895629FD001739FF001829FE00DF11D96
:108C5000649FE00DF11D929FF00D839FF00D749FB6
:108C6000F00D659FF00D9927729FB00DE11DF91F62
:108C7000639FB00DE11DF91FBD01CF0111240895BF
:108C8000991B79E004C0991F961708F0961B881F5E
:108C90007A95C9F780950895AA1BBB1B51E107C0BF
:108CA000AA1FBB1FA617B70710F0A61BB70B881F7C
:108CB000991F5A95A9F780959095BC01CD0108950B
:108CC000A1E21A2EAA1BBB1BFD010DC0AA1FBB1FD0
:108CD000EE1FFF1FA217B307E407F50720F0A21B42
:108CE000B30BE40BF50B661F771F881F991F1A94AF
:108CF00069F760957095809590959B01AC01BD01D9
:108D0000CF01089597FB092E05260ED057FD04D0FC
:108D1000D7DF0AD0001C38F4509540953095219546
:108D20003F4F4F4F5F4F0895F6F7909580957095A0
:108D300061957F4F8F4F9F4F089585FD77C080626B
:108D4000911174C081568A51E0F7089591116EC057
:108D500080538A5028F0865C806281568650B8F72E
:108D600008959111089581548A5108F4805E855ABE
:108D700008959111089581568A5108F480528558BA
:108D80000895FB01DC0105900D920020E1F70895A4
:108D9000FC0105900020E9F7809590958E0F9F1FAC
:108DA0000895FB01DC010D900020E9F71197019077
:108DB0000D920020E1F70895FB01DC0101900D9276
:108DC0000020E1F7089503D0808199270895E0EC11
:108DD000F1E0378537FDFDCF348538603487FC01FD
:108DE000E050F04F0895262FE0ECF1E0378537FD95
:108DF000FDCF3485377F3487378531FF09C036E3AF
:108E0000328738ED34BF31E03387378537FDFDCF0A
:108E100033E33287808391831282248325E3228780
:108E200028ED31E024BF33870196089599278827DC
:068E30000895F894FFCF45
:108E360001000200070008000D000E006461746165
:108E4600006C6574007265616400726573746F729C
:108E56006500676F73756200676F746F006F6E00F1
:108E660072657475726E00696600696E707574005D
:108E76007072696E7400666F72006E657874007346
:108E8600746F7000656E64776800656E6400726565
:108E96006D0064696D0074726F6E0074726F666641
:108EA600007768696C6500656570313600656570C8
:108EB60033320065657000696E62797465003F0043
:108EC6002700656C7365003C3D003E3D003C3E005E
:108ED6003C003E003D00414E44004F5200454F527B
:108EE600002B002D002A002F006D6F64005E0040ED
:108EF6003136004033320040006E6F7400746F00EC
:108F060053544550007468656E00656C7365004780
:108F16004F544F00474F5355420043485224006177
:108F26006273007371727400524E440053474E00D0
:108F36005441420068657834006865783200686597
:108F460078007065656B3136007065656B3332008D
:108F56007065656B0061646472006565703136002A
:108F66006565703332006565700074696D6524004F
:108F7600706F727473004C697374206F6620706F23
:108F8600727473202D2D00200076617273004C6977
:108F96007374206F66207661726961626C657320F6
:108FA6002D2D0020202020002800290020200066EA
:108FB600696C657300556E6B6E6F776E204C495306
:108FC6005420746F7069632E202054727920276CA8
:108FD60069737420706F72747327206F7220276C08
:108FE600697374207661727327206F7220276C690B
:108FF60073742066696C6573272E006D6F6E006C46
:109006006973740072756E006E657700636F6E74B7
:1090160000636C6561720066726565006C6F616401
:109026000073617665006175746F7374006F6666B0
:1090360000656500666C3000666C3100666C320057
:069046004E61BC00004079
:00000001FF
